:020000040000FA
:06000000A9EF3EF0120022
:06100000A9EF3EF0120012
:06100800D6EF27F01200F4
:0610180022EF08F01200B7
:06102A000200A07D0000A1
:1010300000050000E10000009E7D0000BA0E0000E7
:0410400002000000AA
:0C104400D8CFE4FFE0CFE4FFE46EDACF89
:10105000E4FFE2CFDAFFE9CFE4FFEACFE4FFF3CF2A
:10106000E4FFF4CFE4FFE652D9CFE6FFE1CFD9FFAA
:10107000040EE126020EDB6A030EDB6AA4A68CD303
:10108000A4960601FE5101E1A1D0030E526E2D502F
:10109000EA6A510FE96E010EEA22EF50525C30E12C
:1010A0002D50E96EEA6AD890E936EA36690EE926EB
:1010B000010EEA22EECF52F0EFCF53F053C052F0C0
:1010C000536A5250D76E2D50E96EEA6AD890E936CD
:1010D000EA36690EE926010EEA22EECF52F0EFCF92
:1010E00053F05250D66EF28AF294D58E2D50EA6AA1
:1010F000510FE96E010EEA22040EEF6E2D502F6E95
:10110000020E526E2E50EA6A510FE96E010EEA226B
:10111000EF50525C49E12E50E96EEA6AD890E93608
:10112000EA36690EE926010EEA22EE50ED1009E1D9
:101130002E50EA6A510FE96E010EEA22010EEF6E9F
:1011400033D0080E2E5C0CE2070E2E14526E010EE8
:10115000525204E0E846FE0B5206FCE189121AD016
:10116000100E2E5C0CE2070E2E14526E010E52521F
:1011700004E0E846FE0B5206FCE18A120BD0070E93
:101180002E14526E010E525204E0E846FE0B520637
:10119000FCE18B122E50EA6A510FE96E010EEA2231
:1011A000030EEF6E2E502D6E2E2A060E2E5C02E1DF
:1011B000080E04D0130E2E5C03E1160E2E6E67D1BE
:1011C000180E2E5C01E063D12E6A61D10E01005130
:1011D00001E15DD10E01012B0E01AC510E01015D4B
:1011E00001E255D1016B0E01AA51EA6A320FE96E94
:1011F0000E0EEA22EF500E01EA6AAD25E96EAE51FD
:10120000EA22EF6A79907B6A7A6A0E01AA2B0E01B4
:10121000AB510E01AA5D01E3AA6BAA51E96EEA6A1D
:10122000D890E936EA36020EE9260E0EEA22EE5092
:10123000ED1001E12CD1AA51E96EEA6AD890E936A5
:10124000EA364A0EE9260E0EEA22EECF52F0EFCF32
:1012500053F0AA51E96EEA6AD890E936EA36020EEE
:10126000E9260E0EEA22EECF54F0EFCF55F054509F
:10127000521802E15550531801E1CBD0AA51E96E42
:10128000EA6AD890E936EA367A0EE9260E0EEA22A4
:10129000EE50ED1001E1A1D0AA51E96EEA6AD890B2
:1012A000E936EA364A0EE9260E0EEA22EECF54F06F
:1012B000EFCF55F0AA51E96EEA6AD890E936EA36DE
:1012C000020EE9260E0EEA22EE50545C526EEE50EB
:1012D0005558536E020E52C0DBFF030E53C0DBFFA6
:1012E000020EDBCF52F0030EDBCF53F053343BE260
:1012F00052500008000E535436E2020EDBCF52F07B
:10130000030EDBCF53F0AA51E96EEA6AD890E936B2
:10131000EA367A0EE9260E0EEA22EECF54F0EFCF2F
:1013200055F05250545C5350555857E2AA51E96E4B
:10133000EA6AD890E936EA367A0EE9260E0EEA22F3
:10134000EECF52F0EFCF53F0AA51E96EEA6AD8908F
:10135000E936EA36020EE9260E0EEA225250EE2651
:101360005350ED2256D0020EDBCF52F0030EDBCFEE
:1013700053F0526C531E000E5322AA51E96EEA6AD2
:10138000D890E936EA367A0EE9260E0EEA22EECF3A
:1013900054F0EFCF55F05250545C535055581DE265
:1013A000AA51E96EEA6AD890E936EA367A0EE92659
:1013B0000E0EEA22EECF52F0EFCF53F0AA51E96EB3
:1013C000EA6AD890E936EA36020EE9260E0EEA22DB
:1013D0005250EE5E5350ED5A1CD0AA51E96EEA6AA3
:1013E000D890E936EA364A0EE9260E0EEA22EECF0A
:1013F00052F0EFCF53F0AA51E96EEA6AD890E9367D
:10140000EA36020EE9260E0EEA2252C0EEFF53C063
:10141000EDFFAA51EA6A320FE96E0E0EEA22EF5092
:101420000E01EA6AAD25E96EAE51EA22120EEF6EA8
:10143000F29E0E01AA51E96EEA6AD890E936EA36C0
:10144000020EE9260E0EEA22EECF52F0EFCF53F055
:1014500053C052F0536A5250B66EAA51E96EEA6A0E
:10146000D890E936EA36020EE9260E0EEA22EECFD1
:1014700052F0EFCF53F05250B56EF00EB414000995
:10148000B46EF00EB4140909B46E7980F28E000EB9
:10149000D8802154000E22542EE2302A000E312230
:1014A0002150305C2250315826E3306A316A030EF5
:1014B000255C1FE22350EA6A480FE96E010EEA221A
:1014C00080CFEFFF2350EA6A4B0FE96E010EEA224C
:1014D00081CFEFFF2350EA6A4E0FE96E010EEA2238
:1014E00082CFEFFF232A030E235C01E3236A252A20
:1014F00002D0216A226A000ED8802654000E27549A
:1015000019E22B50000816E2322A000E3322265030
:10151000325C275033580EE3326A336A030E2A5C7A
:1015200007E2282A030E285C01E3286A2A2A02D04F
:10153000266A276A2B5000080AE2346A3450040DE8
:10154000F328C26E9E9C9F9C9D8CC280C282050126
:10155000005101E11DD1DE6ADD6ADECF52F0DDCF40
:1015600053F0040E525C000E535801E311D1DECF4C
:10157000E9FFDDCFEAFF010ED890E936EA36E8064A
:10158000FBE1010EE926050EEA22EE50ED1001E125
:10159000D3D0DECFE9FFDDCFEAFF010ED890E936E8
:1015A000EA36E806FBE1110EE926050EEA22EE50C6
:1015B000ED1026E1D9CFE9FFDACFEAFFEE50ED10CA
:1015C00001E18180D9CFE9FFDACFEAFF010EEE1801
:1015D00003E1ED5001E18182D9CFE9FFDACFEAFFE3
:1015E000020EEE1803E1ED5001E18184D9CFE9FF4D
:1015F000DACFEAFF030EEE1803E1ED5001E1818638
:10160000DECFE9FFDDCFEAFF010ED890E936EA36FA
:10161000E806FBE1110EE926050EEA22EECF52F0B4
:10162000EFCF53F0DECFE9FFDDCFEAFF010ED89018
:10163000E936EA36E806FBE1010EE926050EEA2264
:10164000EECF54F0EFCF55F05450521829E15550D9
:10165000531826E1D9CFE9FFDACFEAFFEE50ED10BB
:1016600001E18190D9CFE9FFDACFEAFF010EEE1850
:1016700003E1ED5001E18192D9CFE9FFDACFEAFF32
:10168000020EEE1803E1ED5001E18194D9CFE9FF9C
:10169000DACFEAFF030EEE1803E1ED5001E1819687
:1016A000DECFE9FFDDCFEAFF010ED890E936EA365A
:1016B000E806FBE1110EE926050EEA22EE2A000EED
:1016C000EF22DECFE9FFDDCFEAFF010ED890E93649
:1016D000EA36E806FBE1110EE926050EEA22EECF16
:1016E00052F0EFCF53F0DECFE9FFDDCFEAFF010E7E
:1016F000D890E936EA36E806FBE1090EE926050E40
:10170000EA22EECF54F0EFCF55F0545052183AE1A0
:101710005550531837E1DECFE9FFDDCFEAFF010E68
:10172000D890E936EA36E806FBE1110EE926050E07
:10173000EA22EE6AED6A26D0D9CFE9FFDACFEAFFD6
:10174000EE50ED1001E18190D9CFE9FFDACFEAFF49
:10175000010EEE1803E1ED5001E18192D9CFE9FFCE
:10176000DACFEAFF020EEE1803E1ED5001E18194B9
:10177000D9CFE9FFDACFEAFF030EEE1803E1ED500F
:1017800001E18196DF2A010E01E2E7D6DB2AE5D6E8
:101790000101C45101E0C4079EAC2CD09E9CC450F2
:1017A000566E576E566AC35000015610546E57C09D
:1017B00055F03450060DF3CF52F0F4CF53F0000E35
:1017C0005226010E53222850020D5250F324E96E86
:1017D0005350F420EA6E54C0EEFF55C0EDFF342A9A
:1017E0002B50345C02E39D9C05D03450040DF3284B
:1017F000C26EC282F2A442D0D59EF294F29A040E36
:10180000526E2F50EA6A510FE96E010EEA22EF5034
:10181000525C34E1080E2F5C0DE2070E2F14526E5D
:10182000010E525204E0E846FE0B5206FCE1E81CB1
:1018300089161CD0100E2F5C0DE2070E2F14526E6D
:10184000010E525204E0E846FE0B5206FCE1E81C91
:101850008A160CD0070E2F14526E010E525204E05D
:10186000E846FE0B5206FCE1E81C8B162F50EA6A94
:10187000510FE96E010EEA22020EEF6E040EE15CDA
:1018800002E2E16AE552E16EE552E7CFD9FFE552A7
:10189000E5CFF4FFE5CFF3FFE5CFEAFFE5CFE9FFC2
:1018A000E5CFDAFFE550E5CFE0FFE5CFD8FF100048
:1018B000D9CFE6FFE1CFD9FF020EE126896A92680F
:1018C0002B6A8A6A93688B6A94688C968C94959636
:1018D0009594928E0601010EFD6F0E01BA69BB69E7
:1018E000296A286A2A6A246A236A256A216A226A7E
:1018F000266A276A306A316A326A336A346A7682C3
:101900007680769C769A76887696FA0E776EDF6A7F
:10191000DFCF49F00C0EE76E4918E8AE02D0E7348D
:1019200002D0E750495C36E2010EDB6ADBCF49F0BA
:10193000030EE76E4918E8AE02D0E73402D0E75054
:10194000495C26E2DFCF49F04A6A49BE4A68060E82
:101950004A02F3CF4AF04902F3CF49F0F4504A2645
:10196000000E4926010E4A22010EDBCF4BF04C6AD5
:101970004BBE4C68D8904B364C3649504B24E96EE0
:101980004A504C20EA6EEE6AED6A010EDB2ACED791
:10199000DF2ABED70601F76BF86BF56BF66BF96BB8
:1019A000FA6BFB6BFC6B2D6A2E6A2F6ADF6ADFCF46
:1019B00049F0180EE76E4918E8AE02D0E73402D0BD
:1019C000E750495C1BE2DFCFE9FFEA6AE9BEEA685B
:1019D000D890E936EA36690EE926010EEA22EE6A67
:1019E000ED6ADFCFE9FFEA6AE9BEEA68510EE9264F
:1019F000010EEA22010EEF6EDF2AD9D7D586D59ADD
:101A0000D59CF294F29AF194D08E7694A386A59602
:101A100064EC29F083EC38F0F28EF28C7684020EBE
:101A2000E15C02E2E16AE552E16EE552E7CFD9FFFF
:101A30001200D9CFE6FFE1CFD9FF050EE126020E55
:101A4000DB6A030EDB6A040EDB6A32EC1DF0255004
:101A5000000809E20EEC14F0242A030E245C01E1D4
:101A6000246A2506F4D72A50000809E23EEC14F057
:101A7000292A030E295C01E1296A2A06F4D7200EDF
:101A80000601E76EA819E8AE02D0E73402D0E750AD
:101A9000A85D01E2B7D16550020B01E0B3D1400E61
:101AA000E66E400EE66E020EE66EE6EC36F0E552AD
:101AB000E552E552E76E030EE7CFDBFFDB5000088F
:101AC00001E324D1040EDB6A030EDB50F36E040E37
:101AD000DBCFF4FFF350F45C01E318D1040EDB50CC
:101AE000EA6A400FE96E020EEA22EFCFDFFF05013E
:101AF0005D5141E10D0E496EDF50495C05E00A0E73
:101B00004A6EDF504A5C37E1010E5D6F0601F75106
:101B1000EA6A000FE96E030EEA220D0EEF6EF72B54
:101B2000010EDB6AF751F36E010EDBCFF4FFF350C9
:101B3000F45C1CE2010EDBCFE9FFEA6AE9BEEA6869
:101B4000000EE926030EEA22EF50E66E010EDBCF0F
:101B5000E9FFEA6AE9BEEA68190EE926050EEA22FB
:101B6000E552E750EF6E010EDB2ADCD7D5D906012E
:101B7000F76BF86BBBD01B0EDF5C09E1595107E135
:101B8000010E596F1B0E5A6F5B6B5C6BAFD0590522
:101B90000BE15B0EDF5C08E11B0E5A5D05E15B515A
:101BA00003E15B0E5B6FA2D0590566E1410EDF5C7D
:101BB00063E11B0E5A5D60E15B0E5B5D5DE15A6B9C
:101BC0005B6B5C6B596B010EDB6ADBCFE9FFEA6A8A
:101BD000E9BEEA68000EE926030EEA22EF500D087E
:101BE0001CE0010EDBCFE9FFEA6AE9BEEA68190EE4
:101BF000E926050EEA22EF50E66E010EDBCFE9FF83
:101C0000EA6AE9BEEA68000EE926030EEA22E55216
:101C1000E750EF6E010EDB2AD8D7010EDBCFF7F6C7
:101C20000601F751EA6A000FE96E030EEA22EF6A35
:101C3000270E496E770E4A6E4B6A49C0E6FFE66E84
:101C40004BC0E6FFDBEC3CF0E552E552E552000EFE
:101C5000E66E030EE66E240E496E770E4A6E4B6AF0
:101C600049C0E6FFE66E4BC0E6FFDBEC3CF04C6E95
:101C7000050EE15E4C503AD0080EDF5C1CE1060117
:101C8000F751000818E2F707F751EA6A000FE96E0A
:101C9000030EEA22EF6A210E496E770E4A6E4B6AF6
:101CA00049C0E6FFE66E4BC0E6FFDBEC3CF0E552D8
:101CB000E552E5521BD00D0EDF5C18E00A0EDF5C2A
:101CC00015E0200EDF5C12E305015A6B5B6B5C6B69
:101CD000596B0601F751EA6A000FE96E030EEA221A
:101CE000DFCFEFFF05015D6B0601F72B0601F75112
:101CF000496E4A6A000E491806E1010E4A1803E1CE
:101D00002C86F76BF86B040EDB2ADED62C5001E133
:101D100078D02CA00FD01B0E496E770E4A6E4B6AFE
:101D200049C0E6FFE66E4BC0E6FFDBEC3CF0E55257
:101D3000E552E5522CA20FD0FC0E496E760E4A6E8B
:101D40004B6A49C0E6FFE66E4BC0E6FFDBEC3CF0B9
:101D5000E552E552E5522CA40FD0E00E496E760E06
:101D60004A6E4B6A49C0E6FFE66E4BC0E6FFDBEC0D
:101D70003CF0E552E552E5522CA60FD0C40E496E58
:101D8000760E4A6E4B6A49C0E6FFE66E4BC0E6FF30
:101D9000DBEC3CF0E552E552E5522CA80FD0A50E45
:101DA000496E760E4A6E4B6A49C0E6FFE66E4BC03E
:101DB000E6FFDBEC3CF0E552E552E5522CAC0FD0EF
:101DC000840E496E760E4A6E4B6A49C0E6FFE66E97
:101DD0004BC0E6FFDBEC3CF0E552E552E5522CAEA1
:101DE0000FD06B0E496E760E4A6E4B6A49C0E6FF05
:101DF000E66E4BC0E6FFDBEC3CF0E552E552E55207
:101E00002C6A3FD8050EE15C02E2E16AE552E16E20
:101E1000E552E7CFD9FF1200D9CFE6FFE1CFD9FFD6
:101E2000E652F5C6DFFFDF2A400E496EDF50495CFF
:101E300001E1DF6A0601F651DF5C01E122D806010B
:101E4000F551EA6A000FE96E020EEA22FE0EDBCFC0
:101E5000EFFFF52B400EF55D01E1F56BF651F55DF9
:101E600001E12C84FE0EDBCF49F04A6A49BE4A6884
:101E700049C0F3FF4AC0F4FFE552E552E7CFD9FF6E
:101E80001200D9CFE6FFE1CFD9FFE6520601F551A6
:101E9000F65D3DE00601905105E0DEEC37F017EC11
:101EA0001FF0F8D70601F651D880F55517E2F65124
:101EB000F55DDF6EDFCFE6FFF6514A6A000F496E2F
:101EC000020E4A2249C0E6FF4AC0E6FF46EC37F060
:101ED000E552E552E552F5C6F6F617D0400ED88029
:101EE000F655DF6EDFCFE6FFF6514A6A000F496E06
:101EF000020E4A2249C0E6FF4AC0E6FF46EC37F030
:101F0000E552E552E5520601F66BDEEC37F0E5529C
:101F1000E552E7CFD9FF1200D9CFE6FFE1CFD9FFD5
:101F2000040EE126DE6ADD6A020EDB6A030EDB6A5E
:101F30000601F851EA6A000FE96E030EEA22EF503B
:101F4000E66EE66A34EC3EF0E552E552020EF3CF5F
:101F5000DBFF0601F82BF851496E4A6A000E49185A
:101F600004E1010E4A1801E1F86B020EDB50DE6E4F
:101F7000DD6AF851EA6A000FE96E030EEA22EF50BB
:101F80002C0836E0F851EA6A000FE96E030EEA22E7
:101F9000EF500D082DE0F851EA6A000FE96E030ECC
:101FA000EA22EF50E66EE66A34EC3EF0E552E55286
:101FB000030EF3CFDBFF0601F82BF851496E4A6A96
:101FC000000E491804E1010E4A1801E1F86B020EF7
:101FD000DBCF4BF04BC04CF04B6A030EDB500001E3
:101FE0004B24496E000E4C204A6E49C0DEFFDD6E68
:101FF000000EDFCF3DF0010EDBCF3EF04D0E3D1861
:1020000002E1510E3E1801E1D2D14D0E3D1802E120
:10201000520E3E1801E1C8D1320E3D1802E1530EB6
:102020003E1801E1BED1450E3D1802E1530E3E18A7
:1020300001E1B4D1430E3D1802E1510E3E1801E119
:10204000AAD14B0E3D1802E1430E3E1801E1A0D18A
:102050004C0E3D1802E1420E3E1801E196D1440EAD
:102060003D1802E14E0E3E1801E18CD1490E3D189B
:1020700002E14E0E3E1801E182D1420E3D1802E10E
:10208000510E3E1801E178D14C0E3D1802E1510E7F
:102090003E1801E16ED14C0E3D1802E1530E3E1880
:1020A00001E164D14E0E3D1802E1510E3E1801E1EE
:1020B0005AD14E0E3D1802E1530E3E1801E150D1A7
:1020C000430E3D1802E1530E3E1801E146D14D0E7C
:1020D0003D1802E1450E3E1801E13CD1500E3D187D
:1020E00002E1510E3E1801E132D1500E3D1802E1DD
:1020F000540E3E1801E128D1500E3D1802E1530E56
:102100003E1801E11ED14D0E3D1802E1530E3E185E
:1021100001E114D1470E3D1802E1500E3E1801E1D5
:102120000AD1430E3D1802E1500E3E1801E100D1E4
:10213000490E3D1802E1430E3E1801E1F6D0490E6A
:102140003D1802E1520E3E1801E1ECD0490E3D1857
:1021500002E1530E3E1801E1E2D0530E3D1802E1B8
:10216000430E3E1801E1D8D0530E3D1802E1520E45
:102170003E1801E1CED0530E3D1802E1530E3E1839
:1021800001E1C4D0530E3D1802E1420E3E1801E1B8
:10219000BAD0430E3D1802E1420E3E1801E1B0D024
:1021A000430E3D1802E1520E3E1801E1A6D04F0E3B
:1021B0003D1802E1420E3E1801E19CD0570E3D1839
:1021C00002E14D0E3E1801E193D0520E3D1802E19E
:1021D0004D0E3E1801E18AD0440E3D1802E1500E2A
:1021E0003E1801E181D04F0E3D1802E1500E3E181D
:1021F00001E177D0490E3D1802E1500E3E186EE025
:10220000580E3D1802E1540E3E1865E0540E3D187C
:1022100001E13E505EE0410E3D1801E13E5057E0C5
:10222000560E3D1801E13E5050E0490E3D1801E1C7
:102230003E5049E04F0E3D1801E13E5042E0550E40
:102240003D1802E1430E3E183AE0580E3D1802E1F7
:10225000430E3E1831E0430E3D1801E13E502AE0A6
:10226000520E3D1801E13E5023E0580E3D1802E1A8
:10227000520E3E181AE0030EDB5001E09BD0020E16
:10228000DBCFE6FFE66ADBCFE6FFE66A480E496E83
:10229000760E4A6E4B6A49C0E6FFE66E4BC0E6FF1B
:1022A000DBEC3CF04C6E070EA3D08CEC17F0A2D008
:1022B000D7D8A0D06CD99ED08EEC17F09BD0D4D8B4
:1022C00099D023DA97D0AADA95D0C8DA93D0D6DAA3
:1022D00091D012D98FD08AEC17F08CD001EC16F087
:1022E00089D0A6EC16F086D0A6DB84D062DB82D043
:1022F00022DB80D042EC18F07DD090EC17F07AD041
:1023000040EC18F077D044EC18F074D046EC18F09C
:1023100071D048EC18F06ED04AEC18F06BD04CEC51
:1023200018F068D04EEC18F065D050EC18F062D080
:1023300052EC18F05FD0E3EC18F05CD03FEC2BF0DF
:1023400059D031EC2DF056D0F9EC2CF053D0DEEC16
:102350002CF050D0D5EC2DF04DD0DBEC29F04AD04C
:1023600071EC2EF047D0A1EC2EF044D0BBEC2EF057
:1023700041D0CDEC2EF03ED0E8EC2EF03BD053EC2B
:102380002EF038D064EC2EF035D020EC19F032D09D
:1023900028EC19F02FD005EC2FF02CD06AEC2FF0A0
:1023A00029D0FEEC38F026D0F5EC2FF023D0F6EC57
:1023B0002FF020D0030EDBCFE6FFE66A020EDBCF64
:1023C000E6FFE66A030EDBCFE6FFE66A020EDBCF2E
:1023D000E6FFE66A200E496E760E4A6E4B6A49C0E9
:1023E000E6FFE66E4BC0E6FFDBEC3CF04C6E0B0EFE
:1023F000E15E4C500601F851EA6A000FE96E030EE7
:10240000EA22EF500D080DE02C500BE1520E496E00
:102410004A6ADF50491803E1DE52DD504A1801E0F4
:102420002C8EF7C6F8F6040EE15C02E2E16AE55292
:10243000E16EE552E7CFD9FF12000601FD510FE032
:10244000FC0E496E7C0E4A6E4B6A49C0E6FFE66E92
:102450004BC0E6FFDBEC3CF0E552E552E5521200E2
:1024600058EC0CF01DEF12F0D9CFE6FFE1CFD9FF09
:10247000030EE126E66AD9CFE6FFDACFE6FF010ECA
:10248000E66E62EC1AF0E552E552E552E552E66A74
:10249000D950010FE66E000EDA20E66E020EE66EEF
:1024A00062EC1AF0E552E552E552E5522C501AE181
:1024B000DF0417E1D950010FE96EDACFEAFFEE50E1
:1024C000ED100AE0010E496E4A6ADB50491808E136
:1024D000020EDB504A1804E1010EDBCFFDF601D0FD
:1024E0002C8CABDF030EE15C02E2E16AE552E16EA7
:1024F000E552E7CFD9FF1200D9CFE6FFE1CFD9FFF0
:10250000030EE126020EDB6AE66A1F0EE66E000E7F
:10251000E66E030EE66E62EC1AF0E552E552E55205
:10252000E552E66AD950020FE66E000EDA20E66E3A
:10253000010EE66E62EC1AF0E552E552E552E55204
:102540002C501BE1020EDB500CE11F50201003E168
:10255000216A226A11D076841FC021F020C022F0A7
:102560000BD01F50201003E1266A276A05D076841D
:102570001FC026F020C027F060DF030EE15C02E2FE
:10258000E16AE552E16EE552E7CFD9FF1200D9CFFB
:10259000E6FFE1CFD9FF0A0EE126E66AD9CFE6FFD2
:1025A000DACFE6FF010EE66E62EC1AF0E552E55274
:1025B000E552E552E66AD950010FE66E000EDA20C8
:1025C000E66E010EE66E62EC1AF0E552E552E55257
:1025D000E552E66AD950020FE66E000EDA20E66E8A
:1025E000010EE66E62EC1AF0E552E552E552E55254
:1025F000E66AD950040FE66E000EDA20E66E010E90
:10260000E66E62EC1AF0E552E552E552E552E66AF2
:10261000D950050FE66E000EDA20E66E010EE66E6A
:1026200062EC1AF0E552E552E552E552E66AD950FD
:10263000060FE66E000EDA20E66E010EE66E62EC24
:102640001AF0E552E552E552E552E66AD950070F15
:10265000E66E000EDA20E66E010EE66E62EC1AF00F
:10266000E552E552E552E552E66AD950080FE66EAA
:10267000000EDA20E66E010EE66E62EC1AF0E5520C
:10268000E552E552E552E66AD950090FE66E000EB2
:10269000DA20E66E010EE66E62EC1AF0E552E552C3
:1026A000E552E552E66AD950030FE66E000EDA20D5
:1026B000E66E010EE66E62EC1AF0E552E552E55266
:1026C000E5522C5018E1DF50926E010EDB50936EF4
:1026D000020EDB50946E040EDB50956E050EDB503F
:1026E000966E030EDB500C0805E20C0EF36E030E23
:1026F000F3CFDBFFA2DE0A0EE15C02E2E16AE55203
:10270000E16EE552E7CFD9FF1200D9CFE6FFE1CF66
:10271000D9FF020EE126E66AD9CFE6FFDACFE6FF5F
:10272000010EE66E62EC1AF0E552E552E552E55212
:10273000E76E010EE7CFDBFF2C5066E1010EDB50A8
:1027400002E1DF50896E010EE66ED9CFE6FFDACFE7
:10275000E6FFE66E62EC1AF0E552E552E552E5520C
:10276000E76E010EE7CFDBFF2C504EE1010EDB5090
:1027700002E1DF508A6E010EE66ED9CFE6FFDACFB6
:10278000E6FFE66E62EC1AF0E552E552E552E552DC
:10279000E76E010EE7CFDBFF2C5036E1010EDB5078
:1027A00002E1DF508B6E010EE66ED9CFE6FFDACF85
:1027B000E6FFE66E62EC1AF0E552E552E552E552AC
:1027C000E76E010EE7CFDBFF2C501EE1010EDB5060
:1027D00002E1DF508C6E010EE66ED9CFE6FFDACF54
:1027E000E6FFE66E62EC1AF0E552E552E552E5527C
:1027F000E76E010EE7CFDBFF2C5006E1010EDB5048
:1028000002E1DF508D6E19DE020EE15C02E2E16A48
:10281000E552E16EE552E7CFD9FF12008450E66E33
:10282000E66A8350E66EE66A8250E66EE66A81509A
:10283000E66EE66A8050E66EE66A030E496E760E34
:102840004A6E4B6A49C0E6FFE66E4BC0E6FFDBEC22
:102850003CF04C6E0D0EE15E4C501200040E496EC1
:102860007D0E4A6E4B6A49C0E6FFE66E4BC0E6FF3E
:10287000DBEC3CF0E552E552E5521200D9CFE6FF21
:10288000E1CFD9FFE652DF6A010E496E760E4A6E3D
:102890004B6A49C0E6FFE66E4BC0E6FFDBEC3CF05E
:1028A000E552E552E552DF6A2B50DF5C30E2DFCFC4
:1028B00049F04A6A49BE4A68060E4A02F3CF4AF016
:1028C0004902F3CF49F0F4504A26000E4926010E82
:1028D0004A222950020D4950F324E96E4A50F4204F
:1028E000EA6EEECFE6FFEFCFE6FFFB0E4B6E750E06
:1028F0004C6E4D6A4BC0E6FFE66E4DC0E6FFDBEC6A
:102900003CF04E6E050EE15E4E50DF2ACDD7010E33
:10291000496E7D0E4A6E4B6A49C0E6FFE66E4BC0BB
:10292000E6FFDBEC3CF0E552E552E552E552E552BC
:10293000E7CFD9FF1200D9CFE6FFE1CFD9FF030ED1
:10294000E126E66AD9CFE6FFDACFE6FFE66E62EC73
:102950001AF0E552E552E552E552E66AD950020F07
:10296000E66E000EDA20E66E010EE66E62EC1AF0FC
:10297000E552E552E552E5522C5011E1DECF49F027
:10298000DDCF4AF0000E495C100E4A5807E2DECF58
:10299000E9FFDDCFEAFF020EDBCFEFFF4EDD030ED6
:1029A000E15C02E2E16AE552E16EE552E7CFD9FF70
:1029B0001200D9CFE6FFE1CFD9FF030EE126E66A88
:1029C000D9CFE6FFDACFE6FFE66E62EC1AF0E55209
:1029D000E552E552E5522C5024E1DECF49F0DDCF3F
:1029E0004AF0000E495C100E4A5807E2DECFE9FFBC
:1029F000DDCFEAFF020EEFCFDBFF020EDBCFE6FFFB
:102A0000E66AF10E496E750E4A6E4B6A49C0E6FFE2
:102A1000E66E4BC0E6FFDBEC3CF04C6E050EE15E73
:102A20004C50030EE15C02E2E16AE552E16EE552D0
:102A3000E7CFD9FF1200D9CFE6FFE1CFD9FF030ED0
:102A4000E126E66AD9CFE6FFDACFE6FF050EE66EAD
:102A500062EC1AF0E552E552E552E552E66AD950C9
:102A6000010FE66E000EDA20E66E010EE66E62ECF5
:102A70001AF0E552E552E552E552E66AD950020FE6
:102A8000E66E000EDA20E66E010EE66E62EC1AF0DB
:102A9000E552E552E552E5522C5001E0A8D0020E75
:102AA000DB50010801E2A0D0010EDB50070801E273
:102AB0009BD0410E496EDF50495C1AE1020EDB509B
:102AC0000CE1010EF36EDB5004E0D890F336E8061B
:102AD000FCE1F350F31C921689D0010EF36EDB502B
:102AE00004E0D890F336E806FCE1F35092127ED071
:102AF000420E496EDF50495C1AE1020EDB500CE1D8
:102B0000010EF36EDB5004E0D890F336E806FCE1EA
:102B1000F350F31C93166AD0010EF36EDB5004E001
:102B2000D890F336E806FCE1F35093125FD0430EE1
:102B3000496EDF50495C1AE1020EDB500CE1010ED8
:102B4000F36EDB5004E0D890F336E806FCE1F35076
:102B5000F31C94164BD0010EF36EDB5004E0D890BA
:102B6000F336E806FCE1F350941240D0440E496E6F
:102B7000DF50495C1AE1020EDB500CE1010EF36EEE
:102B8000DB5004E0D890F336E806FCE1F350F31C88
:102B900095162CD0010EF36EDB5004E0D890F3367E
:102BA000E806FCE1F350951221D0450E496EDF5046
:102BB000495C1AE1020EDB500CE1010EF36EDB50B2
:102BC00004E0D890F336E806FCE1F350F31C9616C7
:102BD0000DD0010EF36EDB5004E0D890F336E8061A
:102BE000FCE1F350961202D02C8C01D026DC030EAF
:102BF000E15C02E2E16AE552E16EE552E7CFD9FF1E
:102C00001200D9CFE6FFE1CFD9FF030EE126020E75
:102C1000DB6AE66AD9CFE6FFDACFE6FF050EE66E9D
:102C200062EC1AF0E552E552E552E552E66AD950F7
:102C3000010FE66E000EDA20E66E010EE66E62EC23
:102C40001AF0E552E552E552E5522C5075E1010EBD
:102C5000DB50070856E3410E496EDF50495C0BE13B
:102C6000010EF36EDB5004E0D890F336E806FCE189
:102C7000F35080143FD0420E496EDF50495C0BE1A7
:102C8000010EF36EDB5004E0D890F336E806FCE169
:102C9000F35081142FD0430E496EDF50495C0BE195
:102CA000010EF36EDB5004E0D890F336E806FCE149
:102CB000F35082141FD0440E496EDF50495C0BE183
:102CC000010EF36EDB5004E0D890F336E806FCE129
:102CD000F35083140FD0450E496EDF50495C11E16B
:102CE000010EF36EDB5004E0D890F336E806FCE109
:102CF000F3508414E76E020EE7CFDBFFDB5008E0F1
:102D000002D02C8C19D0010EF36E020EF3CFDBFF34
:102D1000020EDBCFE6FFE66AE80E496E750E4A6EDC
:102D20004B6A49C0E6FFE66E4BC0E6FFDBEC3CF0C9
:102D30004C6E050EE15E4C50030EE15C02E2E16A6E
:102D4000E552E16EE552E7CFD9FF1200D9CFE6FF99
:102D5000E1CFD9FF030EE126E66AD9CFE6FFDACF4D
:102D6000E6FF050EE66EAEDBE552E552E552E552B2
:102D7000E66AD950010FE66E000EDA20E66E010E0B
:102D8000E66EA0DBE552E552E552E552E66AD9501F
:102D9000020FE66E000EDA20E66E010EE66E92DBA2
:102DA000E552E552E552E5522C5001E0A9D0020E61
:102DB000DB50010801E2A0D0010EDB50070801E260
:102DC0009BD0410E496EDF50495C1AE1020EDB5088
:102DD0000CE1010EF36EDB5004E0D890F336E80608
:102DE000FCE1F350F31C891689D0010EF36EDB5021
:102DF00004E0D890F336E806FCE1F35089127ED067
:102E0000420E496EDF50495C1AE1020EDB500CE1C4
:102E1000010EF36EDB5004E0D890F336E806FCE1D7
:102E2000F350F31C8A166AD0010EF36EDB5004E0F7
:102E3000D890F336E806FCE1F3508A125FD0430ED7
:102E4000496EDF50495C1AE1020EDB500CE1010EC5
:102E5000F36EDB5004E0D890F336E806FCE1F35063
:102E6000F31C8B164BD0010EF36EDB5004E0D890B0
:102E7000F336E806FCE1F3508B1240D0440E496E65
:102E8000DF50495C1AE1020EDB500CE1010EF36EDB
:102E9000DB5004E0D890F336E806FCE1F350F31C75
:102EA0008C162CD0010EF36EDB5004E0D890F33674
:102EB000E806FCE1F3508C1221D0450E496EDF503C
:102EC000495C1AE1020EDB500CE1010EF36EDB509F
:102ED00004E0D890F336E806FCE1F350F31C8D16BD
:102EE0000DD0010EF36EDB5004E0D890F336E80607
:102EF000FCE1F3508D1202D02C8C02D01DEC12F0AC
:102F0000030EE15C02E2E16AE552E16EE552E7CFD1
:102F1000D9FF12001DEF12F01DEF12F01DEF12F09D
:102F2000D9CFE6FFE1CFD9FF040EE126E66AD9CF7B
:102F3000E6FFDACFE6FF050EE66EC4DAE552E552AB
:102F4000E552E552E66AD950010FE66E000EDA202E
:102F5000E66E010EE66EB6DAE552E552E552E5524E
:102F6000E66AD950020FE66E000EDA20E66E030E16
:102F7000E66EA8DAE552E552E552E5522C5076E1CC
:102F8000D950020FE96EDACFEAFF720ED880EE5404
:102F90002E0EED5441E3D950020FE96EDACFEAFF6D
:102FA000EE50ED101FE04C684D684E6A2D0EE76E36
:102FB000020EDBCF4FF0030EDBCF50F0E7504F2671
:102FC000000E5022516A4F504C5C496E50504D5883
:102FD0004A6E51504E584B6E020E49C0DBFF030E35
:102FE0004AC0DBFF010EDB50070816E3410E496EB5
:102FF000DF50495C02E1DF6A11D0420E496EDF50BA
:10300000495C02E1080E06D0430E496EDF50495C70
:1030100003E1100EDF6E02D02C8C28D0010EDB50A5
:10302000DF24E96EEA6AD890E936EA36690EE926C5
:10303000010EEA22020EDBCFEEFF030EDBCFEDFF27
:10304000010EDB50DF24EA6A510FE96E010EEA221D
:10305000EF040AE1010EDB50DF24EA6A510FE96E4A
:10306000010EEA22020EEF6E1DEC12F0040EE15C7E
:1030700002E2E16AE552E16EE552E7CFD9FF1200C4
:103080001DEF12F01DEF12F01DEF12F01DEF12F008
:103090001DEF12F01DEF12F01DEF12F01DEF12F0F8
:1030A0001DEF12F0D9CFE6FFE1CFD9FF070EE126E1
:1030B000E66AD9CFE6FFDACFE6FF030EE66E02DA64
:1030C000E552E552E552E552E66AD950020FE66E46
:1030D000000EDA20E66E030EE66EF4D9E552E552F4
:1030E000E552E5522C5065E1DECF01F5DDCF02F56A
:1030F000020EDBCF09F5030EDBCF0AF5040EDB6A07
:10310000030EF36E040EDBCFF4FFF350F45C4FE2DA
:10311000010EE66ED9CFE6FFDACFE6FF030EE66ECC
:10312000D1D9E552E552E552E552E76E050EE7CFFB
:10313000DBFF010EE66ED950020FE66E000EDA20BC
:10314000E66E030EE66EBED9E552E552E552E55253
:10315000E76E060EE7CFDBFF2C502BE1050EDB50B0
:1031600026E1060EDB5023E1040EDB28E96EEA6A55
:10317000D890E936EA36010EE926050EEA22DECFBE
:10318000EEFFDDCFEDFF040EDB28E96EEA6AD89092
:10319000E936EA36090EE926050EEA22020EDBCFF1
:1031A000EEFF030EDBCFEDFF040EDB2AA9D71DECEB
:1031B00012F0070EE15C02E2E16AE552E16EE552CF
:1031C000E7CFD9FF1200D9CFE6FFE1CFD9FFE65212
:1031D000E66AD9CFE6FFDACFE6FF010EE66E72D9D6
:1031E000E552E552E552E5522C500DE1DF5007E083
:1031F000F00E9314936E0501010E006F02D00501CD
:10320000006B1DEC12F0E552E552E7CFD9FF12003A
:10321000D9CFE6FFE1CFD9FFE652DF6AFF0EDF5CD0
:103220000AE2E868E85005E0E80600D000D000D0E7
:10323000F9D7DF2AF3D7E552E552E7CFD9FF1200DD
:10324000F29EF29C6592656AE3DF0FEF00F01200D8
:10325000D9CFE6FFE1CFD9FF100EE126E66AD950BB
:10326000010FE66E000EDA20E66EE66A2BD9E55213
:10327000E552E552E552E66AD9CFE6FFDACFE6FF3E
:10328000010EE66E1FD9E552E552E552E552E66AB7
:10329000D950040FE66E000EDA20E66E020EE66EDE
:1032A00011D9E552E552E552E552E66AD950020FCE
:1032B000E66E000EDA20E66E030EE66E03D9E552E6
:1032C000E552E552E552E66AD9500A0FE66E000E65
:1032D000DA20E66E060EE66EF5D8E552E552E552C6
:1032E000E552E66AD950060FE66E000EDA20E66E69
:1032F000070EE66EE7D8E552E552E552E552E66A7A
:10330000D9500E0FE66E000EDA20E66E040EE66E61
:10331000D9D8E552E552E552E552E66AD9500F0F89
:10332000E66E000EDA20E66E050EE66ECBD8E552AC
:10333000E552E552E552010EDBCF49F04A6A49BE3B
:103340004A6849C0E6FF4AC0E6FFDC0E4B6E750EC8
:103350004C6E4D6A4BC0E6FFE66E4DC0E6FFDBECFF
:103360003CF04E6E050EE15E4E50DFCFE6FFE66AA2
:10337000D00E496E750E4A6E4B6A49C0E6FFE66E86
:103380004BC0E6FFDBEC3CF04C6E050EE15E4C50B2
:10339000040EDBCFE6FF050EDBCFE6FFC40E496E61
:1033A000750E4A6E4B6A49C0E6FFE66E4BC0E6FFFB
:1033B000DBEC3CF04C6E050EE15E4C50020EDBCFB8
:1033C000E6FF030EDBCFE6FFB80E496E750E4A6EC0
:1033D0004B6A49C0E6FFE66E4BC0E6FFDBEC3CF013
:1033E0004C6E050EE15E4C50D9500A0FE96EDACFF3
:1033F000EAFFEECFE6FFEECFE6FFEECFE6FFEFCF40
:10340000E6FFAB0E496E750E4A6E4B6A49C0E6FF89
:10341000E66E4BC0E6FFDBEC3CF04C6E070EE15E67
:103420004C50D950060FE96EDACFEAFFEECFE6FF37
:10343000EECFE6FFEECFE6FFEFCFE6FF9E0E496E42
:10344000750E4A6E4B6A49C0E6FFE66E4BC0E6FF5A
:10345000DBEC3CF04C6E070EE15E4C500E0EDBCF09
:10346000E6FFE66A920E496E750E4A6E4B6A49C0D7
:10347000E6FFE66E4BC0E6FFDBEC3CF04C6E050E63
:10348000E15E4C500F0EDBCFE6FFE66A860E496E1A
:10349000750E4A6E4B6A49C0E6FFE66E4BC0E6FF0A
:1034A000DBEC3CF04C6E050EE15E4C501DEC12F076
:1034B000100EE15C02E2E16AE552E16EE552E7CF0F
:1034C000D9FF1200D9CFE6FFE1CFD9FF090EE126DF
:1034D000080EDB6A0D0E496E0601F851EA6A000F0C
:1034E000E96E030EEA22EF50495C05E1FB0EDB506A
:1034F00044E12C8842D0F851EA6A000FE96E030ECD
:10350000EA22EF502C081FE0FB0EDB501AE1F851C5
:10351000EA6A000FE96E030EEA22EF50E66EE66AF1
:103520005F0E496E750E4A6E4B6A49C0E6FFE66E45
:103530004BC0E6FFDBEC3CF04C6E050EE15E4C5000
:103540002C8A020EE5D1F82BF851496E4A6A000E1A
:10355000491804E1010E4A1801E1F86B0D0E496E9D
:10356000F851EA6A000FE96E030EEA22EF50495C57
:1035700006E1FB0EDB5001E12C88030EC9D12D0EB4
:10358000496EF851EA6A000FE96E030EEA22EF5025
:10359000495C2EE1040E4A6EFE0EDB504A5C28E0C8
:1035A000050E4B6EFE0EDB504B5C22E0FE0EDB0484
:1035B00001E147D1030E496EFE0EDB50495C01E18B
:1035C00040D1070E4A6EFE0EDB504A5C01E139D154
:1035D000010EF36E080EF3CFDBFFF82BF851496EA6
:1035E0004A6A000E491804E1010E4A1801E1F86B1D
:1035F000040E496EFE0EDB50495C11E0050E4A6E6A
:10360000FE0EDB504A5C0BE00A0EE66ED9CFE6FFF9
:10361000DACFE6FF89D9E552E552E55242D0F851BA
:10362000EA6A000FE96E030EEA22EFCF49F0000EBE
:1036300049C0DFFF010EDB6A020EDB6A030EDB6AA4
:10364000050E496EFE0EDB50495C1FE1000EDFCF18
:10365000E6FF010EDBCFE6FF34EC3EF0E552E5522B
:10366000F3CF49F0F4CF4AF04B6A4C6A4AAE02D02D
:103670004B684C6849C0DFFF010E4AC0DBFF020EF9
:103680004BC0DBFF030E4CC0DBFF0601F82BF851EB
:10369000496E4A6A000E491804E1010E4A1801E118
:1036A000F86B080EDB506FE0FE0EDB500FE1D9CF58
:1036B000E9FFDACFEAFFD880800EEE54000EEE5418
:1036C000000EEE54000EEE5401E2BBD0020E496E25
:1036D000FE0EDB50495C0FE1D9CFE9FFDACFEAFFFC
:1036E000D880000EEE54800EEE54000EEE54000E04
:1036F000EE5401E2A6D0060E4A6EFE0EDB504A5C86
:103700000FE1D9CFE9FFDACFEAFFD880000EEE54FF
:10371000000EEE54000EEE54800EEE5401E291D0F5
:10372000D9CFE9FFDACFEAFF040EEECFDBFF050EBB
:10373000EECFDBFF060EEECFDBFF070EEECFDBFF9B
:10374000080EDB5001E196D0040EDBCF3BF0050EF6
:10375000DBCF3CF0060EDBCF3DF0070EDBCF3EF0BB
:103760004068416842684368FCEC3DF0040E37C095
:10377000DBFF050E38C0DBFF060E39C0DBFF070E8E
:103780003AC0DBFF77D0FE0EDB500EE1D9CFE9FF68
:10379000DACFEAFFD8807F0EEE54000EEE54000E12
:1037A000EE54000EEE544DE3FE0EDB040EE1D9CFD5
:1037B000E9FFDACFEAFFD880FF0EEE54000EEE5498
:1037C000000EEE54000EEE543CE3020E496EFE0E67
:1037D000DB50495C0EE1D9CFE9FFDACFEAFFD880B0
:1037E000FF0EEE547F0EEE54000EEE54000EEE541B
:1037F00028E3030E4A6EFE0EDB504A5C0EE1D9CF81
:10380000E9FFDACFEAFFD880FF0EEE54FF0EEE5448
:10381000000EEE54000EEE5414E3060E4B6EFE0E38
:10382000DB504B5C11E1D9CFE9FFDACFEAFFD8805A
:10383000FF0EEE54FF0EEE54FF0EEE547F0EEE54CC
:1038400003E22C8C010E64D0070E496EFE0EDB5095
:10385000495C10E0D9CFE9FFDACFEAFF040EEECFE2
:10386000DBFF050EEECFDBFF060EEECFDBFF070E14
:10387000EECFDBFFFE0EDB50070A38E0010A25E041
:10388000050A16E0010A14E0030A08E0050A06E04A
:10389000010A04E0050A02E0040E3AD0FC0EDBCF78
:1038A000E9FFFD0EDBCFEAFF040EDBCFEFFF2FD0E9
:1038B000FC0EDBCFE9FFFD0EDBCFEAFF040EDBCF12
:1038C000EEFF050EDBCFEDFF22D0FC0EDBCFE9FFD4
:1038D000FD0EDBCFEAFF040EDBCFEEFF050EDBCFE4
:1038E000EEFF060EDBCFEEFF070E0FD0FC0EDBCF98
:1038F000E9FFFD0EDBCFEAFFDFCFEEFF010EDBCFEE
:10390000EEFF020EDBCFEEFF030EDBCFEEFF000E6D
:10391000496E090EE15C02E2E16AE552E16E49504E
:10392000E552E7CFD9FF1200D9CFE6FFE1CFD9FFAB
:10393000020EE126FD0EDBCFE9FFFE0EDBCFEAFF34
:10394000EE6AEE6AEE6AEE6A010EDB6AFC0EDB508E
:10395000F36E010EDBCFF4FFF350F45C62E206017C
:10396000F851EA6A000FE96E030EEA22EFCFDFFF9B
:10397000300EDF5C51E3DF5039084EE3FD0EDBCF44
:10398000E9FFFE0EDBCFEAFFEECF49F0EECF4AF0C3
:10399000EECF4BF0EFCF4CF00A0E406E416A426A18
:1039A000436A49C03BF04AC03CF04BC03DF04CC0BC
:1039B0003EF0FCEC3DF037C049F038C04AF039C069
:1039C0004BF03AC04CF0300EDF5C4D6E4E6A4F6AE1
:1039D000506AE85049264E504A224F504B225050D0
:1039E0004C22FD0EDBCFE9FFFE0EDBCFEAFF49C024
:1039F000EEFF4AC0EEFF4BC0EEFF4CC0EEFF0601EB
:103A0000F82BF851496E4A6A000E491807E1010E79
:103A10004A1804E1F86B02D0000E04D0010EDB2A34
:103A200095D7010E496E020EE15C02E2E16AE552B1
:103A3000E16E4950E552E7CFD9FF12002550E66EFE
:103A4000E66A530E496E750E4A6E4B6A49C0E6FF30
:103A5000E66E4BC0E6FFDBEC3CF04C6E050EE15E23
:103A60004C5012000601A85108E0010E496E655045
:103A7000020B01E0010E495C1BE105016107000E2C
:103A8000625B63510BE16151621111E18C86A00E02
:103A9000616F0F0E626F010E636F12006151621150
:103AA00063E18C96A00E616F0F0E626F636B120064
:103AB000A80509E0020EA85D06E0040EA85D03E07B
:103AC000100EA85D1BE105016107000E625B6351EA
:103AD0000BE16151621111E18C86200E616F4E0E77
:103AE000626F010E636F1200615162113DE18C96AD
:103AF000200E616F4E0E626F636B1200200EA85D88
:103B000033E105016107000E625B63510AE1615117
:103B100062112AE18C86100E616F270E626F010E12
:103B200018D063050AE1615162111EE18C96100EF6
:103B3000616F270E626F020E0CD0020E635D0BE107
:103B40006151621111E18C86A00E616F860E626F69
:103B5000030E636F12006151621106E18C96100E24
:103B6000616F270E626F636B1200D9CFE6FFE1CF62
:103B7000D9FFFE0EDBCF49F0190EE76E4918E8AE0B
:103B800002D0493403D0E750D880495453E3FD0EA6
:103B9000DB5028E0FE0EDBCFE9FFEA6AE9BEEA6807
:103BA000C80EE926050EEA22EF504A6E010E4A526F
:103BB00004E0E846FE0B4A06FCE1496EFE0EDBCF50
:103BC000E9FFEA6AE9BEEA68D890E936EA36960E75
:103BD000E926050EEA22EE50EFCFEAFFE96E4950E2
:103BE000EF1228D0FE0EDBCFE9FFEA6AE9BEEA68F1
:103BF000C80EE926050EEA22EF504A6E010E4A521F
:103C000004E0E846FE0B4A06FCE1E81C496EFE0EA5
:103C1000DBCFE9FFEA6AE9BEEA68D890E936EA361E
:103C2000960EE926050EEA22EE50EFCFEAFFE96E86
:103C30004950EF16E552E7CFD9FF1200D9CFE6FF82
:103C4000E1CFD9FFFE0EDBCF49F0190EE76E491820
:103C5000E8AE02D0493403D0E750D880495453E34A
:103C6000FD0EDB5029E1FE0EDBCFE9FFEA6AE9BE7B
:103C7000EA68C80EE926050EEA22EF504A6E010EE8
:103C80004A5204E0E846FE0B4A06FCE1E81C496E95
:103C9000FE0EDBCFE9FFEA6AE9BEEA68D890E936B2
:103CA000EA36640EE926050EEA22EE50EFCFEAFF6F
:103CB000E96E4950EF1627D0FE0EDBCFE9FFEA6A26
:103CC000E9BEEA68C80EE926050EEA22EF504A6E00
:103CD000010E4A5204E0E846FE0B4A06FCE1496E3A
:103CE000FE0EDBCFE9FFEA6AE9BEEA68D890E93662
:103CF000EA36640EE926050EEA22EE50EFCFEAFF1F
:0E3D0000E96E4950EF12E552E7CFD9FF1200ED
:023D0E00D9CF0B
:103D1000E6FFE1CFD9FFE652A098636A626A0F011D
:103D2000266B020EE66EE66AE66A270EE66E0F0E58
:103D3000E66E8EEC3CF0496E050EE15E49500F01D7
:103D4000160E396F9F0E376F7B0E366FDF6ADF50AE
:103D5000496E4A6A0C0E495C000E4A5810E2DF5068
:103D6000040DF3CFE9FFF4CFEAFF000EE926040EBD
:103D7000EA22EE6AEE6AEE6AEE6ADF2AE8D7658C1E
:103D80000F01386B6598659C62A607D062960601A4
:103D9000BF6BC46BC56BC66BF7D70601010ED86F3E
:103DA000D96FDA6BDB6BCC6BDF6A030EDF5C26E26C
:103DB000EA6ADF34FE0BEA36E96EB50EE926060E36
:103DC000EA22EE6AED6AEA6ADF34FE0BEA36E96E51
:103DD000AF0EE926060EEA22EE6AED6ADF50EA6AC5
:103DE000D00FE96E060EEA22EF6ADF50EA6AD30FBF
:103DF000E96E060EEA22EF6ADF2AD7D70601080E1F
:103E0000B56F040EB66F0F01160E266F0401300E4B
:103E1000026F040E036F400E016F840E006F0601E7
:103E2000A96BA86BE552E552E7CFD9FF1200D9CFB5
:103E3000E6FFE1CFD9FFE65282BE06D0656A0F01E8
:103E4000366B0601A86B88D00601A85110E1656A9F
:103E50000F01366B160E396F9F0E376F7B0E366F64
:103E600065B602D06586FCD70601010EA86FA805CD
:103E70000AE165BA08D0626A0F01366B368136896D
:103E80000601020EA86F6250040B07E00F013651C5
:103E9000040B03E0629411EC25F065B25DD0625032
:103EA000010B09E00F013651010B05E030DF06017F
:103EB000040EA86F62906250100B07E00F0136519C
:103EC000100B03E0FBEC24F0629862AC1AD00F01F7
:103ED00036AD0FD0010EE66EE66A000EE66EE66ABB
:103EE000730EE66EE66AF5EC3BF0496E060EE15E97
:103EF0004950629C0601D65101E0D607D65101E136
:103F0000E2D96250200B06E00F013651200B02E08F
:103F1000E1EC24F06250020B14E00F013651020B69
:103F200010E0010EE66EE66A000EE66EE66AE668EE
:103F30007F0EE66EF5EC3BF0496E060EE15E4950F1
:103F4000636A040E0601E76EA819E8AE02D0E734F2
:103F500002D0E750A85D02E2A1983AD00F0136A73F
:103F600036D0DF6A040EDF5C32E262A630D064CF66
:103F7000CDF60601CD51780BE842E842E842CE6F1B
:103F80006296CDB506D0CE51EA6AD30FE96E060E21
:103F900005D0CE51EA6AD00FE96E060EEA22EF7024
:103FA000CE5103E129EC25F010D0000EE66EE66A52
:103FB000CD0EE66E060EE66E720EE66EE66AF5EC65
:103FC0003BF0496E060EE15E4950DF2ACBD7A1983F
:103FD000E552E552E7CFD9FF1200D9CFE6FFE1CF96
:103FE000D9FF020EE126FD0EDBA407D0E66AFE0E25
:103FF000DBCFE6FFF7D9E552E552FD0EDBA208D094
:10400000010EE66EFE0EDBCFE6FFECD9E552E5527F
:10401000FE0EDB504A6A260F496E0F0E4A2249C037
:10402000DEFF4AC0DDFFDECFE9FFDDCFEAFFFD0E98
:10403000DBCFEFFF020EE15C02E2E16AE552E16EE6
:10404000E552E7CFD9FF1200D9CFE6FFE1CFD9FF84
:10405000020EE126FD0EDB500AE0FE0EEA6ADB34BA
:10406000FE0BEA36E96EB50EE926060E09D0FE0E05
:10407000EA6ADB34FE0BEA36E96EAF0EE926060E7D
:10408000EA22EECFDEFFEDCFDDFFD9CFE9FFDACFB9
:10409000EAFFEE50ED1003E1F36AF46A44D0DECF9C
:1040A000E9FFDDCFEAFF020EE926000EEA22FB0E51
:1040B000DBCFEEFFFC0EDBCFEDFFDECFE9FFDDCF88
:1040C000EAFFEE52FA0EDBCFEFFF400EDECFE9FF44
:1040D000DDCFEAFFE850EF16880EDECFE9FFDDCF37
:1040E000EAFFE850EF12FD0EDB500AE0FE0EEA6A2E
:1040F000DB34FE0BEA36E96EB50EE926060E09D072
:10410000FE0EEA6ADB34FE0BEA36E96EAF0EE926F4
:10411000060EEA22EF74DECF49F0DDCF4AF049C047
:10412000F3FF4AC0F4FF020EE15C02E2E16AE552ED
:10413000E16EE552E7CFD9FF1200D9CFE6FFE1CF1C
:10414000D9FF020EE126FE0EDB5020E1ADC6E9FFED
:10415000AEC6EAFFEE52400EEF6EADC6E9FFAEC648
:10416000EAFF020EE926000EEA22300EEE6E040E81
:10417000ED6EADC6E9FFAEC6EAFF8C0EEF6EB5C6BA
:10418000E9FFB6C6EAFF840EEF6E3BD0FD0EDB50B2
:10419000E8244B6EFE0EDB50040DF3504B24040D4F
:1041A000F3CF49F0F4CF4AF0000E4926040E4A221C
:1041B00049C0DEFF4AC0DDFF840EDECFE9FFDDCF60
:1041C000EAFFE850EF12FD0EDB50E8244B6EFE0EC6
:1041D000DB50040DF3504B24010F040DF3CF49F0D5
:1041E000F4CF4AF0000E4926040E4A2249C0DEFFF1
:1041F0004AC0DDFF840EDECFE9FFDDCFEAFFE850E5
:10420000EF12020EE15C02E2E16AE552E16EE55274
:10421000E7CFD9FF1200D9CFE6FFE1CFD9FF65A8DC
:104220004ED0FE0EEA6ADB34FE0BEA36E96EB50EBE
:10423000E926060EEA22EE50EFCFEAFFE96E400EC5
:10424000EE16EE6AEE6AEE6AFE0EEA6ADB34FE0BEA
:10425000EA36E96EB50EE926060EEA22EE50EFCFF9
:10426000EAFFE96EEE7CFE0EEA6ADB34FE0BEA360C
:10427000E96EB50EE926060EEA22EF74400E496E8D
:10428000FE0EEA6ADB34FE0BEA36E96EB50EE9266D
:10429000060EEA22EE50EFCFEAFFE96E4950EF1624
:1042A000FE0EEA6ADB34FE0BEA36E96EB50EE9264D
:1042B000060EEA22EE50EFCFEAFFE96EEF7CE55200
:1042C000E7CFD9FF12000601D8514DE1010ED86F9A
:1042D000D95149E1010ED96F020EBC5D0DE1B5C6A1
:1042E000E9FFB6C6EAFFEE52EF6AB5C6E9FFB6C609
:1042F000EAFFC80EEF6E1200BC0535E1CF6BABC60E
:10430000E9FFACC6EAFFEE52400EEF6EABC6E9FF26
:10431000ACC6EAFF020EE926000EEA22300EEE6E6F
:10432000040EED6EABC6E9FFACC6EAFF840EEF6E7D
:10433000010ECF6FADC6E9FFAEC6EAFFEE52400EEA
:10434000EF6EADC6E9FFAEC6EAFF020EE926000E2B
:10435000EA22300EEE6E040EED6EADC6E9FFAEC67B
:10436000EAFF800EEF6E12000601DA6BDB6B020EC5
:10437000BC5D18E1ADC6E9FFAEC6EAFFEE52400EE5
:10438000EF6EADC6E9FFAEC6EAFF020EE926000EEB
:10439000EA22380EEE6E040EED6EADC6E9FFAEC633
:1043A000EAFF1DD0C0510401365D0601C151040170
:1043B000375904E236C4C0F637C4C1F6CAD8B5C608
:1043C000E9FFB6C6EAFF020EE926000EEA22380E21
:1043D000EE6E040EED6EB5C6E9FFB6C6EAFFC80E76
:1043E000EF6E1200D9CFE6FFE1CFD9FF020EE12632
:1043F000000EDE6E040EDD6EFD0EDB50E8244B6E0B
:10440000FE0EDB50040DF3504B24040DF4CF4AF0A4
:10441000D9CFE9FFDACFEAFFF350EE264A50ED227A
:10442000DECFE9FFDDCFEAFFEF9EFD0EDB500AE1B4
:10443000FE0EEA6ADB34FE0BEA36E96EAF0EE926C1
:10444000060E09D0FE0EEA6ADB34FE0BEA36E96E90
:10445000B50EE926060EEA22DECFEEFFDDCFEDFF38
:10446000DECFE9FFDDCFEAFFEF9CDECFE9FFDDCF56
:10447000EAFF040EE926000EEA22EF8C020EE15C50
:1044800002E2E16AE552E16EE552E7CFD9FF1200A0
:1044900065980601BFBF2BD0C4AF09D0020EBC6F18
:1044A000DB5101E161DF0601D96BD86B1200ADC6AB
:1044B000E9FFAEC6EAFFEE52400EEF6EADC6E9FF71
:1044C000AEC6EAFF020EE926000EEA22300EEE6EBC
:1044D000040EED6EADC6E9FFAEC6EAFF8C0EEF6EC0
:1044E000B5C6E9FFB6C6EAFF840EEF6E12000401FE
:1044F00030AF0DD00601010EBC6FDA5101E134DF9F
:104500000601D96BD86BD75123E163EF21F0060187
:10451000020EBC6FADC6E9FFAEC6EAFFEE52400E1A
:10452000EF6EADC6E9FFAEC6EAFF020EE926000E49
:10453000EA22300EEE6E040EED6EADC6E9FFAEC699
:10454000EAFF840EEF6ED96BD86BD75101E1BBDE69
:104550001200D9CFE6FFE1CFD9FFE652400EDF6E61
:104560000601C05D000EC1590AE2C0C6DFFFBB51A3
:1045700002E1010E03D0BB0502E1020EBB6FDF506A
:104580004A6AE850C05DC06F4A50C159C16FB5C694
:10459000E9FFB6C6EAFFEE52DFCFEFFF380EC96F74
:1045A000040ECA6FBFB118D0DF502DE0BDC6F6FFB4
:1045B000BEC6F7FFBD2B000EBE230800F550E66E09
:1045C000C9C6E9FFCAC6EAFFC92B000ECA23E552D5
:1045D000E750EF6EDF06E8D7DF5015E0BDC6E9FF14
:1045E000BEC6EAFFBD2B000EBE23EF50E66EC9C665
:1045F000E9FFCAC6EAFFC92B000ECA23E552E750FD
:10460000EF6EDF06E9D7E552E552E7CFD9FF12009A
:10461000D9CFE6FFE1CFD9FF020EE126ABC6E9FF15
:10462000ACC6EAFFEE52EFCFDFFFDFCF49F04950D3
:104630000601C55D000EC65902E2C5C6DFFFDF50A8
:10464000496E4A6AE850C55DC56F4A50C659C66F83
:10465000010EDB6ADF50F36E010EDBCFF4FFF35087
:10466000F45C16E2010EDB50EA6A380FE96E040EC4
:10467000EA22EF50E66EC2C6E9FFC3C6EAFFC22BCC
:10468000000EC323E552E750EF6E010EDB2AE2D79E
:10469000000ED880C555000EC65527E2ADC6E9FF0D
:1046A000AEC6EAFFEE52400EEF6EADC6E9FFAEC6F3
:1046B000EAFF020EE926000EEA22380EEE6E040E24
:1046C000ED6EABC6E9FFACC6EAFFEF50400B06E16A
:1046D000ADC6E9FFAEC6EAFFC80E05D0ADC6E9FF1C
:1046E000AEC6EAFF880EEF6E28D0ADC6E9FFAEC6B3
:1046F000EAFFEE52400EEF6EADC6E9FFAEC6EAFF2E
:10470000020EE926000EEA22300EEE6E040EED6E69
:10471000ADC6E9FFAEC6EAFF840EEF6EC751C81101
:1047200007E005D0C8C6FAFF0601C751F96EFADFE7
:104730000601C49FD75101E1C6DD020EE15C02E231
:10474000E16AE552E16EE552E7CFD9FF1200D9CF19
:10475000E6FFE1CFD9FFE6520601BF8F020EE66EFB
:10476000E66AE66A270EE66E0F0EE66E8EEC3CF009
:10477000496E050EE15E4950DF6ADF50496E4A6AB4
:104780000C0E495C000E4A5810E2DF50040DF3CFC6
:10479000E9FFF4CFEAFF000EE926040EEA22EE6AF2
:1047A000EE6AEE6AEE6ADF2AE8D7658CDF6A030EEE
:1047B000DF5C10E2DF50EA6AD00FE96E060EEA22F3
:1047C000EF6ADF50EA6AD30FE96E060EEA22EF6A5B
:1047D000DF2AEDD7010EE66EE66AE66AAA0EE66EFD
:1047E000060EE66E8EEC3CF0496E050EE15E495019
:1047F000659C0601080EB56F040EB66F000EAB6F18
:10480000040EAC6FABC6ADF6AE6F32C4A9F6A951BB
:1048100002E1100E12D0010EE66EE66AA90EE66EF7
:10482000060EE66E010EE66EE66AF5EC3BF0496EAA
:10483000060EE15E49500601200EA86FE552E552D2
:10484000E7CFD9FF1200800E0401305D58E1060168
:10485000C00EBF6F04013351030A2FE0010A09E0C3
:10486000030A4BE10601E40EBD6F7A0EBE6F120E15
:104870003ED03251F66EF76AD890F636F7366B0EA8
:10488000F6267B0EF7220900F5CFBDF60A00F5CF1C
:10489000BEF6020E0601F76ABD25F66EBE51F7227E
:1048A0000800F5CFC0F6030EF76ABD25F66EBE51BF
:1048B000F7220800F5CFC1F61200030E325D1AE2AE
:1048C0003251F66EF76AD890F636F7366D0EF62648
:1048D0007B0EF7220900F5CFBDF60A00F5CFBEF634
:1048E000BDC6F6FFBEC6F7FF0800F5500601C06F53
:1048F000C16B12000601BF6B12000601BF6B1200F4
:10490000D9CFE6FFE1CFD9FF020EE1260401386BD3
:10491000396B30511F0B020A11E0030A0CE0010A47
:104920003CE10601BF8F040138810601CB0535E16A
:104930000401388332D00601BF8F2FD00601BF8F0C
:10494000040134BF0BD034510F0BE96EEA6AD890E2
:10495000E936EA36AF0EE926060E0AD034510F0BBF
:10496000E96EEA6AD890E936EA36B50EE926060E0F
:10497000EA22EECFDEFFEDCFDDFFDECFE9FFDDCFB8
:10498000EAFFEF50800B09E0DECFE9FFDDCFEAFF61
:10499000EF50040B02E0010E386F0601BFAF07D0E5
:1049A000380EBD6F040EBE6FBF81020EC06F020EC7
:1049B000E15C02E2E16AE552E16EE552E7CFD9FF40
:1049C00012000F0126A115D0ABC6E9FFACC6EAFF65
:1049D000EF5080080DE1B5C6E9FFB6C6EAFFEF501B
:1049E000840806E1ABC6E9FFACC6EAFF8C0EEF6EA9
:1049F0002691629A12000F0136856298658206013F
:104A0000010ECC6F000EE66EE66AE66EE66A750E83
:104A1000E66EE66AF5EC3BF0496E060EE15E495043
:104A200012000601CC6B000EE66EE66AE66EE66AE0
:104A3000740EE66EE66AF5EC3BF0496E060EE15E3A
:104A4000495065920F01369562A402D06294FCD75A
:104A50001200D9CFE6FFE1CFD9FFE65206012D0EB5
:104A6000D66FFD0ECD1553E17E0ECD15E8407F0BC0
:104A7000040DF3CFABF6F4CFACF6000EAB27040E6B
:104A8000AC23ABC6ADF6ACC6AEF6AD75ABC6E9FFB2
:104A9000ACC6EAFFEF503C0BE842E8420D0835E1B6
:104AA000DF6A080EDF5C23E2ABC6E9FFACC6EAFFB3
:104AB000020EE926000EEA22EE50EFCFEAFFE96E81
:104AC000EF50E66EDF50EA6A300FE96E040EEA221C
:104AD000E552E750EF6EABC6E9FFACC6EAFF020E47
:104AE000E926000EEA22EE2AEF22DF2ADAD7ABC649
:104AF000E9FFACC6EAFF020EE926000EEA22300EFC
:104B0000EE6E040EED6E0DD807D03AD805D0FD0E2E
:104B1000CD15040801E159D8E552E552E7CFD9FF98
:104B200012000601BB6BD76BDA6BDB6BCF6BBC6B18
:104B3000B5C6E9FFB6C6EAFFEF9EB575B5C6E9FF93
:104B4000B6C6EAFFEF9EB575ADC6E9FFAEC6EAFF91
:104B5000EF9EBF6BC06BC16BC46BC56BC66B8FD850
:104B6000000EE66EE66AE66EE66A030EE66EE66A3A
:104B7000F5EC3BF0496E060EE15E495048EF22F03D
:104B8000020E0601BC5D02E108EF23F0BC6BCF51C1
:104B90001AE1ADC6E9FFAEC6EAFFEE52400EEF6E77
:104BA000ADC6E9FFAEC6EAFF020EE926000EEA2214
:104BB000300EEE6E040EED6EADC6E9FFAEC6EAFF36
:104BC0008C0EEF6E1200CF6B1200D9CFE6FFE1CF53
:104BD000D9FFE652B5C6E9FFB6C6EAFFEF50400B73
:104BE00001E0010EDF6E0601B575080EA85D0BE150
:104BF00032C438FF0F01385103E00601100E02D015
:104C00000601040EA86FBC0526E1B5C6E9FFB6C6CD
:104C1000EAFF020EE926000EEA22380EEE6E040EBE
:104C2000ED6E97DC020E0601BB5D06E1B5C6E9FF3D
:104C3000B6C6EAFF840E0DD0DF5006E1B5C6E9FF27
:104C4000B6C6EAFFC80E05D0B5C6E9FFB6C6EAFF8C
:104C5000880EEF6E0FD0C4AF0CD0C751C81107E05B
:104C600005D0C8C6FAFF0601C751F96EFADF060182
:104C7000C49FBC6BE552E552E7CFD9FF1200040197
:104C80003051600BE842E842E842E842E84200095D
:104C900001E0120031510C0A50E00B0A3FE00C0A0F
:104CA00031E0010A22E00B0A1EE0020A1CE0030ABE
:104CB00018E0080A10E0010A0CE00F0A08E0030AF5
:104CC00001E012000601BF8F080EA86F120023EF4B
:104CD00024F0A7EF23F00601A90EBD6F060EBE6FEC
:104CE0000CD080EF24F09EEF26F034510601BD6F0A
:104CF000BE6BAA0EBD27060EBE23BF81010EC06F7C
:104D0000BF8F12000601BF8F04013451EA6AAA0F57
:104D1000E96E060EEA2232C4EFFF1200000EE66EC4
:104D2000E66AE66EE66A020EE66EE66AF5EC3BF0CF
:104D3000496E060EE15E495012001200D9CFE6FF1F
:104D4000E1CFD9FF050EE1260401320510E1305113
:104D50001F0B00090CE10601BF8F030E0401315D3A
:104D600004E10601010ECB6F02D00601CB6B0401FA
:104D7000325101E011D130511F0B020801E00CD17A
:104D800034510F0B000901E107D134510F0B020818
:104D900001E202D1200E0601A85D01E0FDD0BF8F27
:104DA000040134BF16D034510F0BE96EEA6AD89073
:104DB000E936EA36AF0EE926060EEA22EECFDEFF2E
:104DC000EDCFDDFF34510F0BEA6AD30FE96E060E0B
:104DD00015D034510F0BE96EEA6AD890E936EA36FD
:104DE000B50EE926060EEA22EECFDEFFEDCFDDFF9F
:104DF00034510F0BEA6AD00FE96E060EEA22020E5A
:104E0000EFCFDBFFD950020FE96EDACFEAFFEF50A8
:104E1000010B03E1000EDF9401D0DF8434BF0BD01F
:104E200034510F0BE96EEA6AD890E936EA36AF0ED4
:104E3000E926060E0AD034510F0BE96EEA6AD890C3
:104E4000E936EA36B50EE926060EEA22DECFEEFF97
:104E5000DDCFEDFF030E315D20E1DECFE9FFDDCFD9
:104E6000EAFFEF50800B11E034BF07D034510F0B35
:104E7000EA6AD30FE96E060E06D034510F0BEA6AC8
:104E8000D00FE96E060EEA22EF82840EDECFE9FF34
:104E9000DDCFEAFFE850EF127FD0DF74DECFE9FF0D
:104EA000DDCFEAFFEF50800B1BE0DECFE9FFDDCF67
:104EB000EAFFEF9EDECFE9FFDDCFEAFFEF8C020EC7
:104EC000E66EE66ADECFE6FFDDCFE6FF050EE66EB4
:104ED000E66AF5EC3BF0496E060EE15E495005D0FE
:104EE000DECFE9FFDDCFEAFFEF8CDF74D950020F90
:104EF000E96EDACFEAFFEF50020B07E1DECFE9FF00
:104F0000DDCFEAFFEF50800B2BE0040134BF07D068
:104F100034510F0BEA6AD30FE96E060E06D03451F6
:104F20000F0BEA6AD00FE96E060EEA22EF923B0EF3
:104F3000496EDECFE9FFDDCFEAFFE850EF16020E43
:104F4000E66EE66ADECFE6FFDDCFE6FF050EE66E33
:104F5000E66AF5EC3BF0496E060EE15E495007D07B
:104F60003B0EDECFE9FFDDCFEAFFE850EF1604018C
:104F700034510F0B4A6A260F496E0F0E4A22030E58
:104F800049C0DBFF040E4AC0DBFF030EDBCFE9FFA5
:104F9000040EDBCFEAFFEF90050EE15C02E2E16A6E
:0C4FA000E552E16EE552E7CFD9FF1200A8
:044FAC00DACFE4FF75
:104FB000E2CFDAFFE9CFE4FFEACFE4FFE6529EA0BA
:104FC0007BD19E908E0ECE6ECF681850196E1A6AE5
:104FD000010E1B6E020E1E5C0EE10101AD51AE1101
:104FE00004E00101AD07000EAE5B0101AD51AE1151
:104FF00001E01B6A09D11E0401E097D01050111086
:105000000AE11250131007E11450151004E1165074
:10501000171001E189D00101B6510BE018A202D0AE
:105020008C8E01D08C9E18A602D08C8A01D08C9ACE
:105030000AD018A202D08C8E01D08C9E18A602D065
:105040008C8A01D08C9A105011101DE00050082459
:10505000006E01500920016E000ED8800054800EB1
:10506000015410E200C000F001C001F0000E005E2B
:10507000800E015A010E1910196E010E1A6E1006DB
:10508000000E115A1B6A125013101DE002500A2420
:10509000026E03500B20036E000ED8800254800E67
:1050A000035410E202C002F003C003F0000E025EDF
:1050B000800E035A040E1910196E010E1A6E120694
:1050C000000E135A1B6A1A502FE00101B65105E079
:1050D00019B08C8C19B48C8804D019B08B8219B497
:1050E0008C880000000000000000000000000000AC
:1050F00000000000000000000000000000000000B0
:10510000000000000000000000000000000000009F
:1051100000000000000000000101B65103E08C9C7B
:105120008C9802D08B928C986FD0030E1E5C33E16A
:105130000601FE5104E0BAC17BF1BBC17CF10E0156
:10514000005112E0B3CE7AFEB4CE7BFEB1CE4AFE61
:10515000B2CE4BFEB7CE32FE0E010251031104E176
:10516000B1CE02FEB2CE03FE0101C75103E0010140
:10517000B36B8A980101AD51AE1104E00101AD0796
:10518000000EAE5B0101AD51AE1101E01B6A0101E1
:10519000010EBC6F39D0040E1E5C36E10601FE51D3
:1051A00004E0B8C17BF1B9C17CF10E01005115E0FA
:1051B000B5CE7AFEB6CE7BFEAFCE4AFEB0CE4BFE6B
:1051C000B7CE32FE0E010251031104E1AFCE02FE52
:1051D000B0CE03FE0E01010E006F0101C75104E0C5
:1051E0000101010EB36F8A880101AD51AE1104E0D7
:1051F0000101AD07000EAE5B0101AD51AE1101E042
:105200001B6A0101BC6B00D01B504AE01E6A1D5096
:1052100047E01C6A040E1C5C3AE21C50E96EEA6A24
:10522000D890E936EA36990EE926010EEA22EECF49
:1052300058F0EFCF59F01C50E96EEA6AD890E93681
:10524000EA36080EE926000EEA2258C0EEFF59C0E1
:10525000EDFF1C50E96EEA6AD890E936EA36A10EF5
:10526000E926010EEA22EECF58F0EFCF59F01C509C
:10527000E96EEA6AD890E936EA36100EE926000EA1
:10528000EA2258C0EEFF59C0EDFF1C2AC3D7A9C1BE
:1052900018F0AAC11EF0ABC1ADF1ACC1AEF11D6AF0
:1052A0008050800B06E00101C35106E08150010BE4
:1052B00003E10101010EC26FE552E5CFEAFFE5CF40
:1052C000E9FFE5CFDAFF1100010E086E096A010E51
:1052D0000A6E0B6A010E0C6E0D6A010E0E6E0F6ADD
:1052E000106A116A126A136A146A156A166A176AD2
:1052F0001D6ACD92CD9ECD9CCD8ACD98CD96CD9474
:105300008E0ECE6ECF68CD809F809E909D809280C5
:105310000F01FE0E486F0F01170E496F8D84969492
:105320008D829692898C929C8D8096908B8294929D
:105330008C9C959C8C9E959E8C9895988C9A959A11
:10534000949E828E0000000000000000000000001B
:10535000000000000000000000000000000000004D
:1053600000000000000000000000948E829E0101F9
:10537000010EC76F8A9893980101010EB36F010166
:10538000010EB66F0601FE6B0E01010E006F0101EA
:10539000010EBC6F0101C16B0101BD6BBE6BBF6B28
:1053A000C06B0101C26B9380F19E0101010EC36FBE
:1053B000939681961200D9CFE6FFE1CFD9FF030E75
:1053C000E126DF6A010EDB6A020EDB6AE66AD9CFEC
:1053D000E6FFDACFE6FF010EE66E62EC1AF0E55268
:1053E000E552E552E552E66AD950010FE66E000E2D
:1053F000DA20E66E030EE66E62EC1AF0E552E55234
:10540000E552E5522C5001E030D1DF0449E1D9509A
:10541000010FE96EDACFEAFFEE50ED100BE10E015D
:10542000006B0601FE6B0101010EC76F01017B6B72
:105430007C6BEFD0D950010FE96EDACFEAFF010E95
:10544000EE180FE1ED500DE10601010EFE6F0E01A9
:10545000006B939201015A0501E0DBD0020E5A6FF6
:10546000D8D00601FE6B9392B3CEE6FFB4CEE6FF32
:10547000040EE66EB1CEE6FFB2CEE6FF010EE66E9A
:1054800079EC39F0496E060EE15E4950000EE66E89
:10549000E66A010EE66E5BDBE552E552E552B9D0F5
:1054A000020EDF5C15E1D950010FE96EDACFEAFF99
:1054B000EE50ED100AE10101010EB66F959E959A2E
:1054C000949295989690959CA4D00101B66BA1D02A
:1054D000040EDF5C07E1010EDBCFB1FE020EDBCF75
:1054E000B2FE97D0050EDF5C07E1010EDBCFAFFE09
:1054F000020EDBCFB0FE8DD0060EDF5C1CE1D95072
:10550000010FE96EDACFEAFF720ED880EE542E0E4C
:10551000ED540AE2720EF36E010EF3CFDBFF2E0E96
:10552000F36E020EF3CFDBFF010EDBCFBAF1020EFA
:10553000DBCFBBF16ED0070EDF5C1CE1D950010F51
:10554000E96EDACFEAFF720ED880EE542E0EED54DB
:105550000AE2720EF36E010EF3CFDBFF2E0EF36E36
:10556000020EF3CFDBFF010EDBCFB8F1020EDBCF73
:10557000B9F14FD0080EDF5C16E1D950010FE96E8A
:10558000DACFEAFF180ED880EE54000EED5407E291
:10559000180EF36E010EF3CFDBFF020EDB6A010E75
:1055A000DBCFABFE36D0090EDF5C16E1D950010F20
:1055B000E96EDACFEAFF060ED880EE54000EED5405
:1055C00007E2060EF36E010EF3CFDBFF020EDB6A7D
:1055D000010EDBCFACFE1DD00A0EDF5C07E1010E31
:1055E000DBCFB3FE020EDBCFB4FE0DD00B0EDF5CC3
:1055F00007E1010EDBCFB3FE020EDBCFB4FE09D014
:105600000C0EDF5C06E1010EDBCFB5FE020EDBCF38
:10561000B6FE0D0EDF5C0EE1D950010FE96EDACF58
:10562000EAFFEE50ED1004E00101010EC36F02D05D
:105630000101C36B0E0EDF5C16E1D950010FE96E5C
:10564000DACFEAFFEE50ED1004E00101010EC76F62
:1056500002D00101C76BBC0503E1B36B8A9803D08C
:10566000010EB36F8A881DEC12F0030EE15C02E2BA
:10567000E16AE552E16EE552E7CFD9FF1200D9CFDA
:10568000E6FFE1CFD9FF0A0EE126020EDB6A030E28
:10569000DB6A040EDB6A050EDB6A060EDB6A070EA8
:1056A000DB6A080EDB6A090EDB6AE66AD9CFE6FF21
:1056B000DACFE6FF030EE66E62EC1AF0E552E55231
:1056C000E552E552E66AD950020FE66E000EDA2086
:1056D000E66E020EE66E62EC1AF0E552E552E55215
:1056E000E552010EE66ED950040FE66E000EDA2088
:1056F000E66E020EE66E62EC1AF0E552E552E552F5
:10570000E5522C5023E1080EDBCFE6FF090EDBCF7C
:10571000E6FF060EDBCFE6FF070EDBCFE6FF040E4B
:10572000DBCFE6FF050EDBCFE6FF020EDBCFE6FFA9
:10573000030EDBCFE6FFDECFE6FFDDCFE6FF10D8BE
:10574000496E0A0EE15E49501DEC12F00A0EE15C52
:1057500002E2E16AE552E16EE552E7CFD9FF1200BD
:10576000D9CFE6FFE1CFD9FF1D50FEE1D950FB0FA5
:10577000E96EFF0EDA20EA6EEE50ED102EE1D95000
:10578000F90FE96EFF0EDA20EA6EEE50ED1025E11A
:10579000D950F70FE96EFF0EDA20EA6EEE50ED10E9
:1057A0001CE1D950F50FE96EFF0EDA20EA6EEE50DB
:1057B000ED1013E10101020EAA6F190E3D6E3E6A53
:1057C000FD0EDBCF42F0FE0EDBCF43F054EC3DF09C
:1057D0003BC0ABF13CC0ACF1EBD0010E0101AB6FB3
:1057E000AC6BA96B8D908B92FB0EDBCF49F0FC0E5E
:1057F000DBCF4AF0800E4A1413E0020EA911A96F04
:105800003D683E68FB0EDBCF42F0FC0EDBCF43F081
:1058100027EC3DF0FB0E3BC0DBFFFC0E3CC0DBFF8A
:10582000F90EDBCF49F0FA0EDBCF4AF00001800E13
:105830004A1414E0080E0101A911A96F3D683E68E1
:10584000F90EDBCF42F0FA0EDBCF43F027EC3DF050
:10585000F90E3BC0DBFFFA0E3CC0DBFFFD0EDBCFD9
:105860004DF0FE0EDBCF4EF04F6A506A190E406EBF
:10587000416A426A436A4DC03BF04EC03CF04FC0A3
:105880003DF050C03EF0FCEC3DF037C04DF038C06C
:105890004EF039C04FF03AC050F0FB0EDBCF49F06C
:1058A000FC0EDBCF4AF04B6A4C6A4AAE02D04B6822
:1058B0004C680F0ED89049364A364B364C36E806BF
:1058C000F9E149C03BF04AC03CF04BC03DF04CC050
:1058D0003EF04DC040F04EC041F04FC042F050C0CD
:1058E00043F05AEC3EF03BC099F13CC09AF1010EF6
:1058F00001019927000E9A23FB0EDBCFA1F1FC0ECC
:10590000DBCFA2F1FD0EDBCF4DF0FE0EDBCF4EF074
:105910004F6A506A190E406E416A426A436A4DC02E
:105920003BF04EC03CF04FC03DF050C03EF0FCECB0
:105930003DF037C04DF038C04EF039C04FF03AC09E
:1059400050F0F90EDBCF49F0FA0EDBCF4AF04B6A8C
:105950004C6A4AAE02D04B684C680F0ED89049365C
:105960004A364B364C36E806F9E149C03BF04AC0AE
:105970003CF04BC03DF04CC03EF04DC040F04EC03E
:1059800041F04FC042F050C043F05AEC3EF03BC0F3
:105990009BF13CC09CF1010E01019B27000E9C2352
:1059A000F90EDBCFA3F1FA0EDBCFA4F1010EAA6F43
:1059B000010E1D6EE552E7CFD9FF1200BCC149F0C0
:1059C0004A6A49BE4A6849C0E6FF4AC0E6FF4E0E31
:1059D0004B6E750E4C6E4D6A4BC0E6FFE66E4DC0C9
:1059E000E6FFDBEC3CF04E6E050EE15E4E501DEF27
:1059F00012F0D9CFE6FFE1CFD9FF020EE126F40E77
:105A0000DE6E010EDD6EE66ED9CFE6FFDACFE6FF81
:105A1000030EE66E62EC1AF0E552E552E552E552ED
:105A20002C5015E10101BC0506E1DECFE6FFDDCF1C
:105A3000E6FFE66A06D0DECFE6FFDDCFE6FF010E29
:105A4000E66E85D8E552E552E5521DEC12F0020EE5
:105A5000E15C02E2E16AE552E16EE552E7CFD9FF8F
:105A60001200D9CFE6FFE1CFD9FF050EE126DF6AAC
:105A7000010EDB6A020EDB6A010EF36E030EF3CF3A
:105A8000DBFFE66AD9CFE6FFDACFE6FF010EE66E6E
:105A900062EC1AF0E552E552E552E552010EE66E6F
:105AA000D950010FE66E000EDA20E66E030EE66EA8
:105AB00062EC1AF0E552E552E552E552010EE66E4F
:105AC000D950030FE66E000EDA20E66E010EE66E88
:105AD00062EC1AF0E552E552E552E552E76E040E2B
:105AE000E7CFDBFF2C5029E1030EDB50070805E26E
:105AF000010EF36E030EF3CFDBFF010EF36E030E08
:105B0000DB5004E0D890F336E806FCE1F350F31CD8
:105B10009314936E030EDB50030F0E01B76F010E4B
:105B2000DBCFE6FF020EDBCFE6FFDFCFE6FF0FD8CD
:105B3000E552E552E5521DEC12F0050EE15C02E281
:105B4000E16AE552E16EE552E7CFD9FF1200D9CF05
:105B5000E6FFE1CFD9FF1D50FEE10E01010E006FFF
:105B6000FE0EDB0403E10101030E02D00101040E6D
:105B7000AA6F190E3D6E3E6AFC0EDBCF42F0FD0EA1
:105B8000DBCF43F054EC3DF03BC0ABF13CC0ACF19B
:105B9000E66AB7CEE6FFB5EC1DF0E552E552010E20
:105BA0001D6EE552E7CFD9FF1200D9CFE6FFE1CF56
:105BB000D9FF050EE126E66AD9CFE6FFDACFE6FF88
:105BC000010EE66E62EC1AF0E552E552E552E5523E
:105BD000E76E040EE7CFDBFFDB502FE12C5059E1DD
:105BE0000101B65124E0DF5000081FE28D90DF0470
:105BF00003E18D848D82898C020EDF5C03E18D844C
:105C00008D82899C030EDF5C03E18D948D82899CDB
:105C1000040EDF5C03E18D848D92899C050EDF5CB0
:105C20000CE18D948D92899C08D08D8006D0DF5038
:105C3000000802E28D9001D08D80010EE66ED950F1
:105C4000010FE66E000EDA20E66E010EE66E62ECE3
:105C50001AF0E552E552E552E552E76E040EE7CF41
:105C6000DBFFDB5014E12C5014E10101B65108E0D8
:105C7000010EDB50000802E28B9209D08B8207D024
:105C8000010EDB50000802E28C9C01D08C8C1DECD4
:105C900012F0050EE15C02E2E16AE552E16EE552C6
:105CA000E7CFD9FF1200FE0E0101BD5DFF0EBE5908
:105CB000FF0EBF59FF0EC05905E2BD2B000EBE23DB
:105CC000BF23C0231DEF12F00101BD51BE11BF1152
:105CD000C01105E0BD07000EBE5BBF5BC05B1DEFE2
:105CE00012F0D9CFE6FFE1CFD9FF050EE126E66A33
:105CF000D9CFE6FFDACFE6FF070EE66E62EC1AF0C8
:105D0000E552E552E552E552E76E040EE7CFDBFFC0
:105D1000DB500BE1DFCFBDF1010EDBCFBEF1020E98
:105D2000DBCFBFF1030EDBCFC0F11DEC12F0050E8F
:105D3000E15C02E2E16AE552E16EE552E7CFD9FFAC
:105D40001200BDC1E6FFBEC1E6FFBFC1E6FFC0C194
:105D5000E6FF450E496E750E4A6E4B6A49C0E6FF76
:105D6000E66E4BC0E6FFDBEC3CF04C6E070EE15EEE
:105D70004C501DEF12F0E66AC10EE66E010EE66EA3
:105D8000010EE66E62EC1AF0E552E552E552E5527C
:105D90002C5001E012001DEF12F0C1C149F04A6A17
:105DA00049BE4A6849C0E6FF4AC0E6FF3E0E4B6E58
:105DB000750E4C6E4D6A4BC0E6FFE66E4DC0E6FFB9
:105DC000DBEC3CF04E6E050EE15E4E501DEF12F026
:105DD000C2C149F04A6A49BE4A6849C0E6FF4AC0A2
:105DE000E6FF380E4B6E750E4C6E4D6A4BC0E6FFEB
:105DF000E66E4DC0E6FFDBEC3CF04E6E050EE15E5C
:105E00004E500101C26B1DEF12F0D9CFE6FFE1CF7A
:105E1000D9FF040EE126DE6ADD6A020EDB6A030E9C
:105E2000DB6AC26AA40EC16E9E9C9F9CC280010167
:105E30000A0EC46FC451FEE1C282C2B2FED7C45082
:105E40004C6E4B6AC3504B24496E000E4C2049C027
:105E5000DEFFDD6E2D0EC26E01010A0EC46FC4514D
:105E6000FEE1C282C2B2FED7C4504C6E4B6AC35030
:105E700000014B24496E000E4C204A6E020E49C0B0
:105E8000DBFF030E4AC0DBFF020EDBCFE6FF030E93
:105E9000DBCFE6FFDECFE6FFDDCFE6FF2C0E496E5F
:105EA000750E4A6E4B6A49C0E6FFE66E4BC0E6FFD0
:105EB000DBEC3CF04C6E070EE15E4C501DEC12F03A
:105EC000040EE15C02E2E16AE552E16EE552E7CFE1
:105ED000D9FF1200D9CFE6FFE1CFD9FF030EE126AB
:105EE000DF6A010EDB6A040EF36E020EF3CFDBFFF6
:105EF000E66AD9CFE6FFDACFE6FF010EE66E62EC86
:105F00001AF0E552E552E552E552010EE66ED9501F
:105F1000010FE66E000EDA20E66E030EE66E62EC0E
:105F20001AF0E552E552E552E5522C5054E1D950B1
:105F3000010FE96EDACFEAFFFF0ED880EE54030EB0
:105F4000ED541EE3010EDBCFC5F1020EDBCFC6F12F
:105F5000CB680101C56BC66FFC0ECA140009CA6E7E
:105F60009D920F0152815293F00EBA140C09BA6E31
:105F70003F0EBA140009BA6E0E010E0ECC6FCA8421
:105F8000DF5023E0C5C149F0C6C14AF0D8904A327B
:105F90004932D8904A3249324950BB6EC5C14BF0A4
:105FA000C6C14CF0040ED8904B364C36E804FBE1E9
:105FB000300E4B16000E4C16CF0EBA1400014B10CB
:105FC000496E4CC04AF0E85003D0BB6ACF0EBA14F9
:105FD000BA6E1DEC12F0030EE15C02E2E16AE552DA
:105FE000E16EE552E7CFD9FF12001200000EE66E17
:105FF000E66AE66EE66A1D50E66EE66A1E0E496EB9
:10600000750E4A6E4B6A49C0E6FFE66E4BC0E6FF6E
:0E601000DBEC3CF04C6E090EE15E4C501200D1
:02601E004BEC49
:1060200035F0FB0EDBCFF3FFDB06F35000090AE08F
:1060300099EC35F0FA0E04EC36F0F3E14A1CF1E18C
:10604000010E01D0000E7AEF35F04BEC35F03B0E2F
:10605000E12402E3E168E652E16E010EDB6A020E22
:10606000DB6AF90EDBCFF6FFFA0EDBCFF7FFFB0E94
:10607000DBCFF8FF0800F550DF6EDF5002E19EEF46
:1060800034F0250EDF5C02E091EF34F0030EDB6AA2
:10609000040EDB6A050EDB6A060EDB6A070EDB6A9E
:1060A000B3EC34F02D0EDF5C0CE02B0EDF5C09E06E
:1060B000200EDF5C06E0230EDF5C03E0300EDF5CC9
:1060C0001AE1DF50300A14E0130A0FE0030A0AE075
:1060D0000B0A05E0060AE4E1030EDB80E1D7030EBC
:1060E000DB82DED7030EDB84DBD7030EDB86D8D75B
:1060F000030EDB88D5D72A0EDF5C1BE1AFEC34F052
:10610000FDEC34F010E0030EDB803D683E68130EBA
:10611000DBCF42F0140EDBCF43F027EC3DF0040E52
:106120003BC0DBFF03D0130EE6EC34F0B3EC34F0ED
:106130000BD0090EDB6A54EC35F003E0C8EC35F007
:10614000FAD7090EE6EC34F0030EDBB0DB982E0E26
:10615000DF5C1BE1B3EC34F02A0EDF5C0BE1AFEC4B
:1061600034F0FDEC34F003E1130E38EC35F0B3EC11
:1061700034F00BD0090EDB6A54EC35F003E0C8ECC8
:1061800035F0FAD7090E38EC35F0680EDF5C07E120
:10619000B3EC34F0680EDF5C1DE1030E18D0740E12
:1061A000DF5C17E07A0EDF5C14E0480EDF5C06E08F
:1061B000540EDF5C03E05A0EDF5C02E1020E07D0F2
:1061C0006C0EDF5C03E06A0EDF5C04E1010E8BEC19
:1061D00035F0C9DBDF506E0A01E17FD31E0A01E111
:1061E00092D1200A01E18FD13F0A01E149D11A0A77
:1061F00001E146D10D0A01E143D1200A01E140D17C
:106200003A0A01E13DD1200A01E13AD1260A01E131
:1062100035D10D0A01E132D11A0A01E1D9D0200AA3
:106220004AE0300A1FE0460A0EE0250A01E083D367
:10623000D950F90FE96EFF0EDA20EA6E010EEE5E1C
:10624000000EEE5AEE5A99EC35F0250EE66E95DB0F
:1062500003E14A1C01E169D395EC35F001E26BD30F
:10626000DB2A69D3080EDB6A040EDB50010806E264
:10627000040EDB045DEC35F0DB508BDB080EDB50ED
:1062800009E0030EDB50010B05E172DB01E04DD3A9
:10629000080EDB6A64DBEFCFDFFF0DEC36F003E1C5
:1062A0004A1C01E142D395EC35F001E3DB2A60DBC7
:1062B00001E141D33AD3070EDB5002080FE1D9ECDC
:1062C00035F0030EA0EC35F00E0EEECFDBFF0F0E17
:1062D000EECFDBFF100EEECFDBFF20D0F70EDBCFD3
:1062E0004CF0F80EDBCF4DF0020E4C5E000E4D5A16
:1062F000F70E4CC0DBFFF80E4DC0DBFF4CC0E9FFD2
:106300004DC0EAFF90EC35F04B6A0E0E49C0DBFF42
:106310000F0E4AC0DBFF100E4BC0DBFF0E0EDBCFB3
:10632000E6FF0F0EDBCFE6FF100EDBCFE6FFB6EC8D
:106330003CF0E552E552E552130E3CC0DBFF140E73
:106340003DC0DBFF060EDB5005E0130ED4EC35F04C
:1063500001E26ADBF8EC35F002E2130E37DBBBEC4E
:1063600035F006E0040ED4EC35F002E2050E2EDB2B
:10637000030EDBB005D0FCDA01E0D7D2080EDB6AF1
:10638000090EDB6A0E0EDBCFF6FF0F0EDBCFF7FF39
:10639000100EDBCFF8FF0800F550DF6EDF5014E081
:1063A000FEEC35F011E20DEC36F003E14A1C01E1A0
:1063B000BCD2BBDB01E3DB2A090EDB2AD9500E0F6E
:1063C000E96E000ECBDBE7D7D3DA01E1B4D2ADD270
:1063D000C6DA110EEECFDBFF120EEDCFDBFF110E92
:1063E000DBCFE6FF120EDBCFE6FFA8EC3CF0E55278
:1063F000E552130EF3CFDBFF140EF4CFDBFF060ED6
:10640000DB5004E0130ED0DB01E20EDBF8EC35F0DC
:1064100002E2130EDBDAAFDB05E0040EC5DB02E2BD
:10642000050ED4DA030EDBB005D0A2DA01E07DD28E
:10643000080EDB6A090EDB6A110EDBCFE9FF120ED4
:10644000DBCFEAFFEFCFDFFFDF5014E0D7DB12E254
:10645000E4DB03E14A1C01E168D267DB01E3DB2AEC
:10646000090EDB2A110EDB2ADBCFE9FF120EE8E36F
:10647000DB2AE6D77DDA01E15ED257D2030EDB8E4E
:10648000070EDB0410E195DB040E5ADB0A0EEECF9B
:10649000DBFF0B0EEECFDBFF0C0EEECFDBFF0D0EA6
:1064A000EECFDBFF6CD0070EDB5003082CE1030EB0
:1064B000DBAE0DD0B2DA020E76DAEFCF49F04A6ADF
:1064C0004B6A4C6A49AE39D04A684B6835D0F70EF2
:1064D000DBCF4AF0F80EDBCF4BF0020E4A5E000E27
:1064E0004B5AF70E4AC0DBFFF80E4BC0DBFF4AC029
:1064F000E9FF4BC0EAFFEFCF49F00A0E49C0DBFFCE
:106500000B0EDB6A38D0070EDB50020809E1030EE0
:10651000DBAE04D059DB4BAE10D00ED055DB0DD026
:10652000030EDBAE12D079DA020E3DDAF9DA4B6AED
:106530004C6A4AAE02D04B684C68E2DA0C0E4BC093
:10654000DBFF0D0E4CC0DBFF1AD0F70EDBCF4BF09C
:10655000F80EDBCF4CF0020E4B5E000E4C5AF70EDD
:106560004BC0DBFFF80E4CC0DBFF4BC0E9FF4CC05B
:10657000EAFFD6DAC5DA0C0EDB6A0D0EDB6A060E10
:10658000DB5005E1010EF36E050EF3CFDBFF150EB8
:10659000DB6A160EDB6AD950370F496E000EDA201F
:1065A0004A6E390E49C0DBFF3A0E4AC0DBFF380E97
:1065B000DB6A080EDB6A0A0EAEDADF50780A12E0F8
:1065C000200A10E0280A0CE0200A0AE03F0A06E050
:1065D0000D0A02E0200A08E1020E05D0080E03D0E1
:1065E000080EDF26100E97DA030EDBBE02D0DB9218
:1065F000DB94DB50800B24E08ADAD890030EEB505A
:10660000000A08E6000EEE5C000EEE58000EEE5892
:10661000000EEE5815E213DA40684168426843689C
:10662000FCEC3DF00A0E37C0DBFF0B0E38C0DBFF81
:106630000C0E39C0DBFF0D0E3AC0DBFF2D0E08D06B
:10664000030EDBA202D02B0E03D0DBA408D0200E59
:10665000F36E170EF3CFDBFF150EDB2A02D0170EF9
:10666000DB6A050EDB5003E1B7D901E189D08A0E60
:10667000496E7D0E4A6E000E4B6E070EDBCF4CF05E
:106680004D6A4E6A4F6A4CC040F04DC041F04EC05A
:1066900042F04FC043F0D3D95AEC3EF04950372472
:1066A000F36E4A503820F46E4B503920F86EF4CF18
:1066B000F7FFF3CFF6FF0800090EF5CFDBFF580E0A
:1066C000DF5C0FE1610EF36E090E7BD90AE3200E49
:1066D000496E090EDBCFE7FF4950E75E090EE7CFB1
:1066E000DBFF070EDBCF49F04A6A4B6A4C6A0FDAD0
:1066F00049C040F04AC041F04BC042F04CC043F0AA
:10670000EECF3BF0EECF3CF0EECF3DF0EFCF3EF0E2
:106710005AEC3EF03EC0EDFF3DC0EDFF3CC0EDFF4A
:106720003BC0EFFF390EDBCFE9FFDB063A0EDBCFD4
:10673000EAFF01E2DB06090EDBCFEFFF150EDB2AD5
:106740004BD995E1030EDBA61DD06F0EDF5C06E191
:10675000C1D918E3150EDB285BDA14D0780EDF5CA4
:1067600009E0580EDF5C06E0620EDF5C03E0420EDB
:10677000DF5C08E1020EF36E160EF3CFDBFF02D0F2
:10678000150EDB6A030EDB50100B0EE0040EDBCFA0
:1067900049F0050EDB50D880495406E2060EDB5066
:1067A00003E1040EDB5034DA95D90AE2050EDBCFA3
:1067B000E7FF150EDB50E75E050EE7CFDBFF02D0EB
:1067C000050EDB6A040EDBCF49F0160E45D9D880E2
:1067D000495414E2160EDBCFE6FF150EDBCFE6FFC1
:1067E000040EDBCFE6FF050EDB50E552E75CE55219
:1067F000D880E754E552D880E7545FD9030EDB50C8
:10680000010B0BE1080EDB5008E0B2D801E08DD09F
:10681000080EDB50BED8080EDB6A170EDB5007E00F
:1068200088D9170EF1D903E14A1C01E17ED0160E7A
:10683000DB5016E07ED9300EE66E9FD802E14A1C8E
:1068400074E077D9DFCFE6FFBAEC3DF0E552E552D0
:10685000E552F4CF4AF00001F31C02E14A1C65E066
:10686000050EDBCF49F0160EDB50D880495409E203
:10687000050EDBCFE7FF160EDB50E75E050EE7CF18
:10688000DBFF300EE66E050ECBD94FE1390EDB2A69
:10689000DBCFE9FF3A0E01E3DB2ADBCFEAFF090E8B
:1068A000EFCFDBFFDB500EE044D9090EADD902E19A
:1068B0004A1C3BE0390EDB2ADBCFE9FF3A0EEDE361
:1068C000DB2AEBD755D831E1160EDBCFE6FF080EF9
:1068D000C3D8E552E7245DD82ED0070EDB50030A5B
:1068E0001CE0010A14E0030A07E07BD9DBCFEEFFCE
:1068F000020EDBCFEDFF1FD0F5D84E6A4CAE02D0B2
:106900004D684E682CD8BCD84EC0EEFF14D0EAD8E3
:106910004CBE4D6824D8B4D80ED063D9DBCFEFFF7E
:106920000AD07BD905E14A1C03E1F368F46810D072
:10693000FCD801E3DB2A79D93AEF30F0010EDBCF46
:1069400049F0020EDBCF4AF049C0F3FF4AC0F4FF22
:106950003B0EE15C02E2E16AE552E16ECBD029D95F
:10696000020EA0EF35F061D90800F550DF6E12007D
:10697000200EE66E080E10EF36F0BAEC3DF0E55250
:10698000E552E552F3CF49F0F4CF4AF00001F31C91
:106990001200496E4A6AD950010F4DD94950EE266E
:1069A0004A50ED2212004D5E000E4E5AF70E4DC0B9
:1069B000DBFFF80E4EC0DBFF4DC0E9FF4EC0EAFF23
:1069C0001200DBCFF4FFF350F45C1200DB50E76EF3
:1069D000040EE7CFDBFF12000A0EDBCF49F00B0EEF
:1069E000DBCF4AF00C0EDBCF4BF00D0EDBCF4CF0C3
:1069F00049504A104B104C101200130EEECFDBFF23
:106A0000140EEDCFDBFF130EDBCF49F0140EDBCFFE
:106A10004AF00001800E4A141200F70EDBCF4DF051
:106A2000F80EDBCF4EF01200050EDB50E66ED950AB
:106A3000130F01D9E552E750EE6EED6A12000A0E0F
:106A4000DBCF3BF00B0EDBCF3CF00C0EDBCF3DF091
:106A50000D0EDBCF3EF01200DBCFE6FF150EDBCFD5
:106A6000E6FF050EDB50E552E724E552E72412006D
:106A7000DB50CED8010EF36E060EF3CFDBFF120013
:106A8000EE50EFCFEAFFE96E4BC0EEFF4CC0EEFFD9
:106A90004DC0EEFF1200D9CFE6FFDACFE6FFE1CF1F
:106AA000D9FFE2CFDAFF1200DFCFE6FFE66A48EC5B
:106AB0003EF0E552E552F3501200E76E080EE7CFC4
:106AC000DBFF1200EECF49F0EECF4AF0EFCF4BF0F4
:106AD0004C6A1200050EDBCF49F0150EDB50D88052
:106AE00049541200010EDBCF4BF0020EDBCF4CF00D
:106AF0004D6A1200E552E5CFDAFFE7CFD9FF120069
:106B00000A0E49C0DBFF0B0E4AC0DBFF1200D95052
:106B10000A0F1BEF36F0F36E070EF3CFDBFF120008
:106B2000EECF49F0EFCF4AF01200010EDB2A020E41
:106B30001200FC0EDBCFE6FFFD0EDBCFE6FF1200FE
:106B4000495E000E4A5AF70E49C0DBFFF80E4AC0F4
:106B5000DBFF49C0E9FF4AC0EAFF1200DA20EA6E13
:106B6000EF2AEECFF6FF000EEF22EECFF7FFEF2277
:106B7000EECFF8FF1200040EDBCFE6FF130EDB5062
:106B8000E552E75C9ADFDB5004DF060EDB501200B3
:106B9000090EDB500A0DF350DF24D00FE76E090E0B
:106BA000E7CFDBFFB3EF34F0DB50F36E050EE1EF20
:106BB00034F0F70EDBCF49F0F80EDBCF4AF01200CD
:106BC000DFCFE6FFBDEF34F028DF030EECDE62EF2F
:106BD00035F00FEC30F0E552E552E552E552000990
:106BE0001200BDDEEE50EFCFEAFFE96E010E12009B
:106BF000130EDB50F36E040EE1EF34F0040EDB50A5
:106C0000F36E090EE1EF34F0DBCFE6FFBDEF34F0B9
:106C1000E76E050EE7CFDBFF12008BDFE0EF35F00C
:106C2000DBCFE6FF86DFE9EF35F0D950F90FE96EEB
:106C3000FF0EAEEF35F0E96E000EDA20EA6E1200BC
:106C4000040130511F0B010801E012003051600BAC
:106C5000E842E842E842E842E842010801E0120066
:106C6000345103E0340501E012003151220A31E0D1
:106C7000030A24E0010A15E0210A0DE0010A01E0FF
:106C800012000601A00EBD6F060EBE6F080EC06F8B
:106C9000C16BBF8121D00601A00EBD6F060EBE6F75
:106CA0001BD036C4C5F637C4C6F60601880EC26FBF
:106CB000060EC36FC76BC86BC48F12000601880E27
:106CC000BD6F060EBE6F070EC06FC16BC10EBF6FEA
:106CD000120032C49BF60601BF8F12000601886BBA
:106CE0004B0E896F8A6B8B6B8C6B8D6B080E8E6F66
:106CF0008F6B1A0EE66E010EE66EEDEC1FF0E5529C
:106D0000E5521E0EE66E020EE66EEDEC1FF0E55249
:106D1000E552400EE66E080EE66E060EE66EE66A78
:106D2000020EE66E24EC20F0496E050EE15E49503D
:106D3000F3CF97F6F4CF98F60601996B9A6B906BA8
:106D40001200D9CFE6FFE1CFD9FFFD0EDBCF3DF03A
:106D5000FE0EDBCF3EF0050E3D1801E13E5002E095
:106D6000000E30D0FB0EDBCF49F0FC0EDBCF4AF03B
:106D700006019751491816E198514A1813E1400E3F
:106D8000E66E080EE66E060EE66EE66A020EE66E29
:106D900024EC20F0496E050EE15E4950F3CF97F6E2
:106DA000F4CF98F6FB0EDBCF49F0FC0EDBCF4AF0B8
:106DB00006019951491805E19A514A1802E1906B70
:106DC000956B010EE552E7CFD9FF1200D9CFE6FF50
:106DD000E1CFD9FF06018F6B9751981102E1000EA8
:106DE00008D097C6E9FF98C6EAFFEF50800B01E094
:106DF000010E000945E1FC0EDBCF49F097C6E9FF23
:106E000098C6EAFFEE52EF50D880495408E297C680
:106E1000E9FF98C6EAFFEE52FC0EEFCFDBFF8F6B67
:106E2000FC0EDB508F5D19E28F51EA6A080FE96EA4
:106E3000060EEA22EF50E66E8F51E76EFD0EDBCFB5
:106E4000E9FFFE0EDBCFEAFFE750E926000EEA225B
:106E5000E552E750EF6E8F2BE3D7400EE66E080E3B
:106E6000E66E060EE66EE66A020EE66E24EC20F092
:106E7000496E050EE15E4950F3CF97F6F4CF98F6D0
:106E800006018F51E552E7CFD9FF1200D9CFE6FFB7
:106E9000E1CFD9FF060190510CE1FD0EDBCF91F659
:106EA000FE0EDBCF92F6FC0EDBCF95F6010E966F51
:106EB000906FE552E7CFD9FF1200D9CFE6FFE1CFBF
:106EC000D9FF030EE126060190512DE1DF6AFD0E88
:106ED000DBCF3DF0FE0EDBCF3EF0DE523DC0DEFFED
:106EE0003EC0DDFFDD52DF2ADF50496E4A6AFF0EE9
:106EF000491802E14A500BE0010EDBCFE9FFDB2A23
:106F0000020EDBCFEAFF01E3DB2AEF50ECE1FD0EDE
:106F1000DBCF91F6FE0EDBCF92F6DFCF95F60601C2
:106F2000010E966F906F030EE15C02E2E16AE5529A
:106F3000E16EE552E7CFD9FF1200D9CFE6FFE1CFEE
:106F4000D9FF030EE126060190512EE1DF6AFD0E06
:106F5000DBCF3DF0FE0EDBCF3EF0DE523DC0DEFF6C
:106F60003EC0DDFFDD52DF2ADF50496E4A6AFF0E68
:106F7000491802E14A500CE0010EDBCFF6FFDB2A94
:106F8000020EDBCFF7FF01E3DB2A0800F550EBE14F
:106F9000FD0EDBCF91F6FE0EDBCF92F6DFCF95F63E
:106FA0000601966B010E906F030EE15C02E2E16A4E
:106FB000E552E16EE552E7CFD9FF1200D9CFE6FFE7
:106FC000E1CFD9FF020EE126060199519A1102E1A3
:106FD000000E08D099C6E9FF9AC6EAFFEF50800B71
:106FE00001E0010E000901E084D0030E905D01E193
:106FF000906B905101E17DD0020E905D16E1E66A42
:10700000000EE66EE66A010EE66E020EE66E24ECF7
:1070100020F0496E050EE15E4950F3CF99F6F4CFAA
:107020009AF60601030E906F64D0900562E1400E5F
:10703000496E4A6A9551495C000E4A5803E2400E77
:10704000DF6E02D095C6DFFFDF50955D956F480E6D
:10705000936F060E946F010EDFCFDBFF965116E1A2
:10706000010EDB5028E091C6F6FF92C6F7FF08003C
:10707000F55093C6E9FF94C6EAFFEF6E932B000E1E
:107080009423912B9223010EDB06EAD7010EDB50ED
:1070900012E091C6E9FF92C6EAFFEF5093C6E9FFFE
:1070A00094C6EAFFEF6E932B000E9423912B92234C
:1070B000010EDB06EBD70601955107E1400EDF5CC0
:1070C00002E1020E01D0030E906FDFCFE6FF480E03
:1070D000E66E060EE66E010EE66E020EE66E24EC1D
:1070E00020F0496E050EE15E4950F3CF99F6F4CFDA
:1070F0009AF6020EE15C02E2E16AE552E16EE552C7
:06710000E7CFD9FF1200E9
:0A710600D9CFE6FFE1CFD9FFE65232
:107110000E01006B016BAA6BDF6A180EDF5C2AE2BE
:10712000EA6ADF34FE0BEA36E96E020EE9260E0E3D
:10713000EA22EE6AED6ADF50EA6A320FE96E0E0E5D
:10714000EA22EF6AEA6ADF34FE0BEA36E96E4A0E9B
:10715000E9260E0EEA22EE6AED6AEA6ADF34FE0BD9
:10716000EA36E96E7A0EE9260E0EEA22EE6AED6A3A
:10717000DF2AD3D70E01C60EAD6F0E0EAE6F3F0ED7
:1071800079140009796ECF0E79140009796E79822D
:107190007B6A7A6A79900F0152815293F00EB4148F
:1071A0000909B46E0E01080EAB6F030EAC6F200E12
:1071B000B16F4E0EB26F800EAF6F3E0EB06F040E09
:1071C000B76F0601FE6B93920E01010E006F900ED9
:1071D000B36F010EB46F900EB56F010EB66F000E57
:1071E000E66EE66A010EE66EA7EC2DF0E552E5527A
:1071F000E552E552E552E7CFD9FF1200D9CFE6FFBD
:10720000E1CFD9FF060EE126DF6A010EDB6A020E2E
:10721000DB6A030EDB6A040EDB6A050EDB6AE66AD4
:10722000D9CFE6FFDACFE6FF010EE66E62EC1AF088
:10723000E552E552E552E552010EE66ED950010FD6
:10724000E66E000EDA20E66E030EE66E62EC1AF0D1
:10725000E552E552E552E552010EE66ED950030FB4
:10726000E66E000EDA20E66E010EE66E62EC1AF0B3
:10727000E552E552E552E552010EE66ED950040F93
:10728000E66E000EDA20E66E030EE66E62EC1AF091
:10729000E552E552E552E5522C5021E1DF50180845
:1072A00004E3030EDB50180802E22C8C18D0040E05
:1072B000DBCFE6FF050EDBCFE6FF030EDBCFE6FFFD
:1072C000010EDBCFE6FF020EDBCFE6FFDFCFE6FFEE
:1072D00010D8496E060EE15E49501DEC12F0060E04
:1072E000E15C02E2E16AE552E16EE552E7CFD9FFE7
:1072F0001200D9CFE6FFE1CFD9FFE652FE0EDB50F8
:1073000052E10E01006BDF6ADFCF49F0180EE76E25
:107310004918E8AE02D0E73402D0E750495C01E3F7
:10732000F9D0DFCFE9FFEA6AE9BEEA68D890E9362A
:10733000EA367A0EE9260E0EEA22EE6AED6ADFCF11
:10734000E9FFEA6AE9BEEA68D890E936EA364A0E09
:10735000E9260E0EEA22EE6AED6ADFCFE9FFEA6A5D
:10736000E9BEEA68320EE9260E0EEA22EF6ADFCFA6
:10737000E9FFEA6AE9BEEA68D890E936EA36020E21
:10738000E9260E0EEA22EE6AED6ADFCF49F04A6A7C
:1073900049BE4A68AD514924E96EAE514A20EA6EB1
:1073A000EF6ADF2AB1D7D950FC0FE96EFF0EDA2061
:1073B000EA6EEE50ED103FE1FE0EDB04EA6A320F9A
:1073C000E96E0E0EEA22EF500E01EA6AAD25E96E73
:1073D000AE51EA22EF6AFE0EDB04E96EEA6AD8904B
:1073E000E936EA367A0EE9260E0EEA22EE6AED6AF0
:1073F000FE0EDB04E96EEA6AD890E936EA364A0EF8
:10740000E9260E0EEA22EE6AED6AFE0EDB04EA6A57
:10741000320FE96E0E0EEA22EF6AFE0EDB04E96E11
:10742000EA6AD890E936EA36020EE9260E0EEA221A
:10743000EE6AED6A6FD0FE0EDB04496E0E01AB51B1
:10744000495C68E2FB0EDB50180864E3FB0EDB507E
:10745000070802E10101C76BE66AFB0EDBCFE6FF1E
:107460001EEC1EF0E552E552E66AFB0EDBCFE6FFAE
:10747000B5EC1DF0E552E5520E01010E006FFE0E57
:10748000DB04E96EEA6AD890E936EA367A0EE92634
:107490000E0EEA22F90EDBCFEEFFFA0EDBCFEDFF88
:1074A000FE0EDB04E96EEA6AD890E936EA364A0E47
:1074B000E9260E0EEA22FC0EDBCFEEFFFD0EDBCF3F
:1074C000EDFFFE0EDB04EA6A320FE96E0E0EEA22D1
:1074D000FB0EDBCFEFFFFE0EDB04E96EEA6AD8900D
:1074E000E936EA36020EE9260E0EEA22EE50ED10DB
:1074F00011E1FE0EDB04E96EEA6AD890E936EA365D
:10750000020EE9260E0EEA22FC0EDBCFEEFFFD0E88
:0E751000DBCFEDFFE552E552E7CFD9FF1200C9
:02751E00514DCD
:107520002C25692C25692C25690A0D002530346924
:107530002C253034690D0A002531690D0A002530EB
:1075400033690D0A00253031306C750D0A00256451
:107550000A0D005374617475733D25690D0A00218D
:1075600035204572723A204E65656420636F6D6DFB
:1075700061206E6578742C20666F756E643A2027E2
:107580002563270D0A00506172616D383D25630D3A
:107590000A00506172616D373D25630D0A0050612C
:1075A00072616D363D256C750D0A00506172616D1A
:1075B000353D256C640D0A00506172616D343D25C6
:1075C000750D0A00506172616D333D25640D0A002E
:1075D000506172616D323D25640D0A005061726127
:1075E0006D313D25640D0A0050492C2531750D0A79
:1075F000004D522C253033750D0A002C2530347582
:10760000004100492C253033692C253033692C2565
:107610003033692C253033692C253033690D0A004D
:107620002138204572723A20556E6B6E6F776E204E
:10763000636F6D6D616E642027256325633A253283
:1076400058253258270D0A002138204572723A20F9
:10765000556E6B6E6F776E20636F6D6D616E64201B
:107660002725633A253258270D0A00213720457215
:10767000723A204578747261207061726D61746530
:10768000720D0A002136204572723A20496E7661E9
:107690006C696420706172616D7465722076616CD2
:1076A00075650D0A002134204572723A204D6973C8
:1076B00073696E6720706172616D6574657228739D
:1076C000290D0A002133204572723A205258204277
:1076D0007566666572206F76657272756E0D0A004A
:1076E0002132204572723A205458204275666665F0
:1076F00072206F76657272756E0D0A002131204519
:1077000072723A2043616E2774207374657020741E
:1077100068617420666173740D0A002130200D0ABF
:10772000002008002573001B5B421B5B314B1B5B79
:03773000304700DF
:0C77340005D817EC1FF019EC0DF0FBD786
:10774000D9CFE6FFE1CFD9FF020EE1260F0148694C
:107750004969600ED36E9B8C580EDE6E020EDD6E94
:10776000DFCF49F0DF06010EDBCF4AF001E2DB0696
:1077700049504A10F5E1948E58EC0CF087EC1EF05D
:10778000020EE15C02E2E16AE552E16EE552E7CF0A
:10779000D9FF1200120012001200120020EF36F082
:1077A00012006EEF36F00601CB051EE10601CC0596
:1077B0001BE1F1DF65920601CC6B0E01100EB86F74
:1077C0000E0EB96FB807000EB95BB851B911FAE1E6
:1077D0006584080EB86F070EB96FB807000EB95B65
:1077E000B851B911FAE165941200D9CFE6FFE1CFA3
:1077F000D9FFFD0EDBCF3DF0FE0EDBCF3EF0050ED8
:107800003D1801E13E5036E0E8683D1802E17F0E88
:107810003E182FE0030E3D1801E13E5028E0020E15
:107820003D1801E13E5021E0010E3D1801E13E50BE
:107830001AE0740E3D1801E13E5013E0750E3D183C
:1078400001E13E500CE0730E3D1801E13E5005E0B1
:10785000720E3D180FE13E500DD09EDF0BD09ADF27
:1078600009D099DF07D09DDF05D09ADF03D096DFDE
:0E78700001D093DF010EE552E7CFD9FF1200E1
:02787E002A0ED0
:10788000F66E100EF76E000EF86E05010900F55049
:10789000E66F0900F550E76F03E1E66701D03DD0E0
:1078A0000900F550E16F0900F550E26F0900F5504D
:1078B000E36F09000900F550E96E0900F550EA6E22
:1078C000090009000900F550E46F0900F550E56F63
:1078D00009000900F6CFE8F5F7CFE9F5F8CFEAF5AA
:1078E000E1C5F6FFE2C5F7FFE3C5F8FF0501E45384
:1078F00002E1E55307E00900F550EE6EE407F8E217
:10790000E507F9D7E8C5F6FFE9C5F7FFEAC5F8FFCF
:0C7910000501E607000EE75BBFD7120080
:04791C00FE0EE3CFA9
:10792000E9FFFF0EE3CFEAFFE9CFF3FFEACFF4FF71
:10793000FB0EE35003E1FC0EE35009E0FB0EE3060F
:1079400002E2FC0EE306FD0EE350EE6EF1D71200EC
:10795000FE0EE3CFE9FFFF0EE3CFEAFFF36AF46A1E
:10796000EE5203E0F34AF42AFBD71200FF0EE3CFF6
:10797000F8FFE552FF0EE3CFF7FFE552FF0EE3CF2E
:10798000F6FFE552E66AE66AE66A0900F55209E0A2
:10799000FD0EE32A05E1FE0EE32A02E1FF0EE32AD3
:1079A000F4D7FD0EE3CF3CF0FE0EE3CF3DF0FF0E2B
:0679B000E3CF3EF01200DF
:0A79B600D9CFE6FFDACFE6FFE1CFFC
:1079C000D9FFE2CFDAFFE652E652E652E652D9504C
:1079D000FB0F496EFF0EDA204A6E49C0DEFFDD6EF6
:1079E000DECFE6FFDDCFE6FFFB0EDBCFE6FFFC0ED2
:1079F000DBCFE6FFFD0EDBCFE6FFBACEE6FFBBCE68
:107A0000E6FF25EC30F0496E070EE15C02E2E16A28
:107A1000E552E16E4950020EF3CFDBFF030EF4CFC7
:107A2000DBFF020EDBCF49F0030EDBCF4AF049C08B
:107A3000F3FF4AC0F4FF040EE15C02E2E16AE552A2
:0E7A4000E16EE552E5CFDAFFE7CFD9FF120085
:027A4E003EC038
:107A500048F03DC047F03D504202F4CF3CF0F3CF38
:107A60003BF03E504302F4CF3EF0F3CF3DF04202F4
:107A7000F3503C26F4503D22E86A3E224750430230
:107A8000F3503C26F4503D22E86A3E2243AE4DEFCF
:107A90003DF047503D5E48503E5A48AE000C4250C3
:107AA0003D5E43503E5A000C3DC047F03D504202FF
:107AB000F4CF3CF0F3CF3BF03E504302F4CF3EF026
:107AC000F3CF3DF04202F3503C26F4503D22E86AE9
:107AD0003E2247504302F3503C26F4503D22E86AD0
:047AE0003E22000C36
:0C7AE4001201000202000040D80492FDD4
:107AF00082010102000109024300020100C03209B3
:107B00000400000102020100052400100104240207
:107B10000205240600010524010001070581030870
:107B2000000209040100020A0000000705020240E9
:107B300000000705820240000004030904180353F3
:107B400000630068006D0061006C007A004800610D
:107B5000007500730016034500690042006F007451
:107B60000042006F00610072006400F67A397B3DCC
:037B70007B557BC7
:0C7B7400D9CFE6FFDACFE6FFE1CFD9FF62
:107B8000E2CFDAFFFB0EDBCF49F0FC0EDBCF4AF091
:107B90000001800E4A141AE1FB0EDBCFE9FFFC0E58
:107BA000DBCFEAFFEECFF3FFEDCFF4FFEE2A000EBE
:107BB000EF22F3CFE9FFF4CFEAFFFD0EDBCFEFFFBB
:107BC000EF504A6AF36E4AC0F4FF10D0FB0EDB5050
:107BD000FE0806E1FD0EDBCFE6FFB7EC3EF005D078
:107BE000FD0EDBCFE6FF0CEC0FF0E552E552E5CFE2
:087BF000DAFFE7CFD9FF120014
:087BF8003B504002F3CF37F0CF
:107C0000F4CF38F04102F3503826000EF420396EDC
:107C10003B504202F3503926000EF4203A6E3B509E
:107C20004302F3503A263C504002F3503826F450B9
:107C30003922000E3A223C504102F3503926F450CA
:107C40003A223C504202F3503A263D504002F35053
:107C50003926F4503A223D504102F3503A263E5024
:087C60004002F3503A26120025
:087C6800FF0EE124E96EFF0E9E
:107C7000E220EA6EEDCFF4FFEFCFF3FFF46607D01A
:107C8000600EF36404D07B0EF36001D0F39A12000F
:107C9000F36AF46AFF0EE124E96EFF0EE220EA6E59
:107CA000ED6607D02F0EEF6404D03A0EEF6001D0DE
:047CB000F32A1200A1
:0C7CB4003A6A396A386A376A200EE76EB7
:107CC000D8903B363C363D363E3637363836393638
:107CD0003A364050375C415038584250395843503A
:107CE0003A5809E34050375E4150385A4250395AA9
:0C7CF00043503A5A3B2AE72EE4D712001A
:047CFC004F4B0D0AD3
:107D0000000D0A004542427631335F616E645F6167
:107D1000626F7665204542204669726D77617265B3
:107D20002056657273696F6E20322E312E350D0A22
:017D30000052
:0E7D3200C00EF36E00EE00F00E0E01D812002F
:107D4000EA6002D0EE6AFCD7F350E9601200EE6AF6
:027D5000FCD75E
:0E7D52001DEE00F02DEE00F0F86A369C3FECBE
:0E7D60003CF0CEEC3EF09AEC3BF0FBD712006C
:027D6E00FF0E06
:107D7000E350ADBA04D0B06AAC8EAD8A949CADA28B
:0A7D8000FED7AE6EF36EF46A120037
:067D8A00303132333435C4
:0B7D90003637383961626364656600B5
:027D9C001200D3
:027D9E00FEFFE6
:107DA00000000000000000000000000000000000D3
:107DB00000000000000000000000000000000000C3
:107DC00000000000000000000000000000000000B3
:107DD00000000000000000000000000000000000A3
:107DE0000000000000000000000000000000000093
:107DF0000000000000000000000000000000000083
:107E000000000000920F920F920F930F930F930FA9
:107E1000930F930F930F930F930F940F940F940F4F
:107E2000940F940F940F940F940F950F950F950F37
:107E3000950F950F950F890F890F890F8A0F8A0F5C
:107E40008A0F8A0F8A0F8A0F8A0F8A0F8B0F8B0F68
:107E50008B0F8B0F8B0F8B0F8B0F8B0F8C0F8C0F50
:107E60008C0F8C0F8C0F8C0F000105000102030496
:107E700005060700010203040506070203040506C0
:017E800007FA
:00000001FF
